:020000040800F2
:10000000001800208B6A0008396A0008016B00089C
:100010003D6A00083F6A0008416A000800000000CD
:10002000000000000000000000000000436A00081B
:10003000456A000800000000476A0008FD0D00083E
:100040004B6A00084D6A00084F6A0008516A0008B0
:10005000536A0008556A0008576A0008596A000880
:100060005B6A00085D6A00085F6A0008616A000850
:10007000636A0008656A0008676A0008696A000820
:100080006B6A00086D6A00086F6A0008716A0008F0
:10009000736A0008756A0008776A0008796A0008C0
:1000A0007B6A00087D6A00087F6A0008710E0008FC
:1000B000836A0008856A0008876A0008D961000819
:1000C0009023DB05802252049A61024B04221A60BD
:0800D0007047C046181500201E
:1000D80033230349034A0A60013B002BFBD17047D5
:0800E80000300040AAAA00004C
:1000F0002E4A91698023DB010B4393619023DB053A
:100100001A682B490A401A601968802292030A4330
:100110001A60284A1168284801401160106880213F
:10012000890101431160596A244801405962586AA3
:100130008021490001435962136A21490B4013622F
:10014000204B214A1360214A1360214B1B68392B35
:1001500027D01CD8132B26D0263B5A1E93415B4236
:100160001C4A13401C4A944663441C4A93818023D2
:100170009B025360002393602C33136013680121AA
:100180000B431360164B802212051A607047603BC8
:100190005A1E93415B42134A1340134A94466344E8
:1001A000E3E7124BE1E7124BDFE7C04600100240E5
:1001B000FFFFEFFF00040048FFEFFFFFFFF0FFFF2E
:1001C000FFFFFFF00411002000150020FC140020A8
:1001D00020150020BFFCFFFFE204000000380140B2
:1001E00000E100E019EEFFFF88130000410300006A
:0401F000C40900003E
:1001F40004498022CB691A42FCD080B2014B188595
:080204007047C04600380140BC
:10020C0010B50400074B1B68002B04D0064B1B6871
:10021C00002B03D110BDFFF7E7FFF7E7200006F036
:0C022C0029F8F7E7081500202C1400202A
:1002380010B504004A4B1868C3434A4A1168CA43B8
:100248000140013100D170E0474901200860190CD4
:10025800464801601B041B0C45480360002902D175
:10026800424944480860002B02D1414B4249196079
:10027800D107C91706230B400A3340490B60404990
:100288000B6013065B0E3F490B60002C4CD05305E6
:100298009B0F3D490B601304DB0E04333B490B6095
:1002A800120C3B4B1A603B4B1B68DB431A04120CC5
:1002B80039490A601B0C394A1360394A1468E44307
:1002C8002204120C802109018A4201D935490A43C6
:1002D80035490A60002B2DD1344B354C3548191956
:1002E80004CBD2430A608342F9D1334C33481919FD
:1002F80004CBD2430A608342F9D103F079FF264B3D
:100308001B68002B07D09023DB051B8A5B0502D4F2
:10031800214B00221A600D20FFF774FF04F01AFB2E
:100328001D4B1B68002B15D110BD04F03DF9002CA6
:10033800E3D1F9E702F0B2FB02F036FC240C80238B
:100348001B019C4201D9174B1C431D4B1C6002F03A
:1003580085FCC1E7013B1B4A136003F057FCE3E748
:10036800007400080474000810150020BC14002054
:100378001415002083040000405700007C1400205E
:10038800501400202015002058140020601400206C
:100398005C14002008740008B8140020941400208D
:1003A8000C7400080000FFFF781400201074000887
:1003B8000094FF17007A00081088FF1700800008D3
:0803C8007414002070140020E1
:1003D000F0B5C64600B586B001A9294B0A0013CB7B
:1003E00013C203CB03C2274B01221A60264B002203
:1003F0001A6005F033F9254A254B1A60254B9846BB
:10040000254F234E254D06E02B68002B13D1204BA2
:100410001B68002B0FD043461F6034689442F3D012
:10042000A3059B0D1E4922008B42EDD12E20FFF724
:10043000EDFE2200E8E701A806F087FB174B1B68DA
:10044000002B0CD06F20FFF7E1FE6B20FFF7DEFEE4
:10045000C82000F089F806B080BCB846F0BD652021
:10046000FFF7D4FE7220FFF7D1FE7220FFF7CEFE19
:100470006F20FFF7CBFE7220FFF7C8FEE8E7C0460B
:1004800008630008C014002028140020B80B0000E6
:100490000415002000300040AAAA00002C140020FF
:0404A000FF03000056
:1004A40010B5254B1B68002B22D1234B32221A6036
:1004B400224B234A1A60234B1B68002B19D0013BA3
:1004C400204A1360002B14D09023DB051B8A9B0564
:1004D4000ED51D4B1B68002B0AD01C4B1B68002B30
:1004E40006D01B4B1B685A1C132B08D0184B1A60E0
:1004F40010BD9023DB05802252009A61E4E7144B7F
:1005040000221A60134B1B68002BF1D1124B1A60A6
:10051400124B1B681F2B09D0114B1B68002BE7D112
:10052400FFF754FF0D20FFF76FFEE1E70B4B0B3293
:100534001A60FFF7DBFDEFE70C15002000300040E8
:10054400AAAA000018150020BC14002014150020CD
:10055400101400202C140020081500202015002061
:04056400C01400209F
:1005680010B5054B1860002805D01C00FFF796FF52
:0C0578002368002BFAD110BD1C150020D8
:10058400F8B5D1490122CB681A42FCD1CE4B1B6984
:100594001B0604D5CC4BCD4A5A60CD4A5A60CA4B8F
:1005A4001A6902210A431A61CA4A5A611A693E3118
:1005B4000A431A6119000122CB681A42FCD1C24BCA
:1005C400DB689B0604D5C04AD36820210B43D36063
:1005D400BD4B1A6902218A431A611A6901390A4317
:1005E4001A61BD4B1B68DB43BA4A1380B64901222A
:1005F400CB681A42FCD1B44BDB689B0604D5B24AE3
:10060400D36820210B43D360B44B1B68DB43B44A4B
:100614001380AD490122CB681A42FCD1AA4BDB6896
:100624009B0604D5A84AD36820210B43D360AD4B65
:100634001B685B00FF221A40AB4B1B680A3B591E28
:100644008B411A43A94B1B685B02C021C9000B40B4
:100654001A43A74B1B68043BDB061B0C1343DB4309
:10066400A44A138098490122CB681A42FCD1964BC4
:10067400DB689B0604D5944AD36820210B43D360DE
:100684009D4B1B68DB439D4A13808F490122CB6835
:100694001A42FCD18C4BDB689B0604D58A4AD3688A
:1006A40020210B43D360964B1B68DB43954A138090
:1006B40085490122CB681A42FCD1834BDB689B0637
:1006C40004D5814AD36820210B43D3608E4B1B6829
:1006D400DB438E4A13807C490122CB681A42FCD149
:1006E400794BDB689B0604D5774AD36820210B43FA
:1006F400D360874B1B68DB43864A1380724901220F
:10070400CB681A42FCD1704BDB689B0604D56E4A59
:10071400D36820210B43D3607F4B1B68DB437F4AA4
:10072400138069490122CB681A42FCD1664BDB680D
:100734009B0604D5644AD36820210B43D3607848D0
:10074400784C241A604B01222025774F02E00430B4
:10075400B8421AD006190168C9433180D9680A42DF
:10076400FCD1D9680D4202D0D9682943D960016807
:10077400C943090C7180D9680A42FCD1D9680D4279
:10078400E5D0D9682943D960E1E74F4B1A690121C3
:100794008A431A61654A664911601A6902210A434B
:1007A4001A61644A5A611A693E310A431A6119008E
:1007B4000122CB681A42FCD1434BDB689B0604D56B
:1007C400414AD36820210B43D3603F4B1A6902216D
:1007D4008A431A611A6901390A431A61524801228B
:1007E4002025554F02E00430B8421AD0061901689A
:1007F400C9433180D9680A42FCD1D9680D4202D07C
:10080400D9682943D9600168C943090C7180D96842
:100814000A42FCD1D9680D42E5D0D9682943D96090
:10082400E1E74648464C241A274B01222025454F30
:1008340002E00430B84219D006190168C943318076
:10084400D9680A42FCD1D9680D4202D0D96829433B
:10085400D9604188C9437180D9680A42FCD1D968FA
:100864000D42E6D0D9682943D960E2E7164B1A69EC
:1008740001218A431A612D4A2D4911601A69022106
:100884000A431A61304A5A611A693E310A431A61AD
:1008940019000122CB681A42FCD10B4BDB689B0682
:1008A40004D5094AD36820210B43D360064B1A6947
:1008B40002218A431A611A6901390A431A61012221
:1008C4002025224F47E0C04600200240230167450F
:1008D400AB89EFCD0074000814150020BC1400206F
:1008E40002740008201500207C14002058140020F5
:1008F40060140020047400085C14002006740008CE
:10090400B814002008740008941400200A74000825
:10091400781400200C740008741400200E7400086D
:100924001008002010740008000C00200030004063
:10093400AAAA000000780008000E0020100200207F
:10094400007A000810040020007C00081008002031
:100954000430B84219D006190168C9433180D968F6
:100964000A42FCD1D9680D4202D0D9682943D96022
:100974004188C9437180D9680A42FCD1D9680D42C3
:10098400E6D0D9682943D960E2E7064B1A69012108
:100994008A431A611A697F310A431A610A20FFF7F0
:0809A400E1FDF8BD0020024056
:1009AC0070B5041E00DA9CE0092C00D893E0632C8F
:1009BC0000D881E0FA239B009C426ED3534B9C429F
:1009CC005AD9534B9C4248D9524B9C4236D9524B24
:1009DC009C4224D9514B9C4212D9514B9C4200D978
:1009EC0084E05049200006F063FB05004D492000CF
:1009FC0006F0E9FA0C0028003030C0B2FFF700FC1A
:100A0C004949200006F054FB05004749200006F038
:100A1C00DAFA0C0028003030C0B2FFF7F1FB434982
:100A2C00200006F045FB05004049200006F0CBFAFB
:100A3C000C0028003030C0B2FFF7E2FB3C4920002C
:100A4C0006F036FB05003A49200006F0BCFA0C0013
:100A5C0028003030C0B2FFF7D3FB3649200006F037
:100A6C0027FB05003349200006F0ADFA0C002800E6
:100A7C003030C0B2FFF7C4FBFA218900200006F029
:100A8C0017FB0500FA218900200006F09CFA0C00E7
:100A9C0028003030C0B2FFF7B3FB6421200006F011
:100AAC0007FB05006421200006F08DFA0C002800DD
:100ABC003030C0B2FFF7A4FB0A21200006F0F8FA90
:100ACC0005000A21200006F07EFA0C0028003030C8
:100ADC00C0B2FFF795FB20003030C0B2FFF790FB9F
:100AEC0070BD2D20FFF78CFB64425DE7124920009E
:100AFC0006F0DEFA05001049200006F064FA0C003E
:100B0C0028003030C0B2FFF77BFB6AE70F270000EC
:100B1C009F8601003F420F007F969800FFE0F5058D
:100B2C00FFC99A3B00E1F5058096980040420F0002
:0C0B3C00A08601001027000000CA9A3BB0
:100B480070B58CB006AD124B2A0013CB13C213CB71
:100B580013C26C460F4B220043CB43C243CB43C264
:100B68000D20FFF74FFB280005F0EBFF3520FFF7BE
:100B780049FB2E20FFF746FB2420FFF713FF200038
:100B880005F0DFFF0D20FFF73DFB0CB070BDC04640
:080B98001C630008346300082F
:100BA00010B5544B5969802292020A435A6159691F
:100BB0008022D2020A435A619022D2050023136098
:100BC0004D490B604D48D0604D48C860D0684D4CD1
:100BD0002040D060116821401160106880214902D6
:100BE00001431160802149009161474ACE3911606B
:100BF000464A1360464A1360464A1360464A4749CC
:100C00001160474A47491160474A1360474A1360D9
:100C1000474A13600A2247490A6047490A60474A1F
:100C20001360474B0B221A60464B474A1A60474BEA
:100C30001868FA21890006F041FA013880235B0424
:100C400098420DD2424A50604248036A1B021B0A76
:100C5000C02109060B43036200239360073313602E
:100C60000A20FFF781FC3C4C3C4B23603C4BA360CB
:100C70000220FFF779FC022363600220FFF774FC77
:100C8000384B23600020FFF7D7FA0220FFF76CFCF7
:100C9000FFF72EFA0220FFF767FCFFF755FF02204F
:100CA000FFF762FC304B00221A609023DB051B8AA1
:100CB0009B0507D5184B1B68002B03D0184B1B68EE
:100CC000934213D1294805F040FF0D20FFF792FA17
:100CD0000120FFF7B1FA264C03F0F6FA01F030F9E3
:100CE0002368002BF8D002F0F9FFF5E7FFF770FB5F
:100CF000EEE7C0460010024000040048AAAA0AA479
:100D0000AAAAAAAAFFFFFCFF0C15002018150020B4
:100D10001C15002004150020BC14002083040000D2
:100D2000141500204057000028140020C014002093
:100D3000101500207C1400205014002008150020FD
:100D40002015002068140020A1B0B9120C02002068
:100D500010E000E000ED00E00030004055550000DC
:100D6000FFFF0000CCCC00002C140020D06E000847
:040D70004414002007
:100D740010B5FFF795FB0F4B1B680F4A126893429F
:100D840016D05A1C0B490A601B78802000021843B5
:100D94000A4B1B689A4208D09023DB058022520438
:100DA4009A61074B04221A6010BD064A0A60F3E7F1
:100DB4000020F9E7FC1400200015002008020020A0
:080DC4001815002004110020A5
:100DCC0010B5094B1B68002B05D1084B1B68002084
:100DDC00002B05D010BD05F02FF80028F5D0F9E751
:100DEC00FFF7C2FFF6E7C0462C14002008150020C0
:100DFC00164B1B68002B02D0013B144A1360144B9A
:100E0C001B68002B02D0013B114A1360114B1B686D
:100E1C00002B02D0013B0F4A13600F4B1B68002BB9
:100E2C0002D0013B0C4A13600C4B1B68002B02D008
:100E3C00013B0A4A13600A490A6853035A40530C8F
:100E4C0053405A0153400B607047C0460C150020AC
:100E5C001C150020041500208814002054140020B8
:040E6C0068140020E6
:100E700010B51A4BDB699B062BD5184B9B8C9BB28C
:100E8000174A1268002A1AD1FF321A40022A0FD0DC
:100E9000042A11D0134A11680B70136801331360D0
:100EA000114A1268934214D10E4B104A1A6010E096
:100EB0000F4A02211160EDE700F052FD09E0094AF6
:100EC00011680B70136801331360074A126893426C
:100ED00000D010BD034B054A1A60FAE70038014004
:100EE0000815002000150020080200200411002031
:040EF0004814002082
:100EF400024A202311680B431360704798140020A2
:100F0400064A1368043B1360054A0C32934204D228
:100F1400044A042311680B431360704764140020CF
:080F24005C130020981400206A
:100F2C00084B1A68111D1960074B5433994202D2B1
:100F3C00136853607047054A042311680B43136010
:100F4C00F8E7C046641400205C13002098140020BD
:100F5C00044B19680A1F1068096811601B68186037
:080F6C007047C0466414002028
:100F7400034A1368191D11601A1F12685A607047DA
:040F840064140020D1
:100F8800074A1368190008390868043B1B680B6096
:100F98001368191F1B680B60136818607047C046F8
:040FA80064140020AD
:100FAC00074A13681968181F006818601368181F1F
:100FBC00083B1B6803601368083B19607047C04608
:040FCC006414002089
:100FD0000C4B19680A680C4BCB1A9B109B1A042BFC
:100FE00006D4002A0AD092008A1A13680B60704750
:100FF000064A042311680B431360F8E70439014BD8
:101000001960F4E7641400205C1300209814002099
:1010100030B5144B1A681168134BD31A9B105B1A26
:10102000042B19D4043A0F4B1A60012913D9012358
:101030005B1A9B009D580222521A9200094C2368A9
:1010400098589B18043B1860013904320029F6D1E6
:10105000044B1B681D6030BD044A042311680B4318
:101060001360F8E7641400205C130020981400203B
:10107000F0B5144B1A681568134BD31A9B105B1B01
:10108000042B19D4043A17680E4B1A60012D12D99B
:101090006E1E0422524200211C00236898589B189F
:1010A00058600131043AB142F7D101235D1B054B71
:1010B0001B68AD00EF50F0BD044A042311680B43D8
:1010C0001360F8E7641400205C13002098140020DB
:1010D000054B1A68111F12680868844662440A604A
:0C10E0001A68043A1A607047641400207B
:1010EC00024B1A68136801331360704764140020B4
:1010FC00054B1A68111F12680868821A0A601A6870
:0C110C00043A1A607047C04664140020CA
:10111800024B1A681368013B13607047641400207F
:10112800044B1A681368002B00DB70475B4213609E
:08113800FBE7C046641400202F
:1011400010B50F4B1B681A68D117501848401F285C
:1011500009DC191F0A4C2160002A0BDB0B0009680F
:101160009140196010BD074A8023DB0011680B43D2
:101170001360F7E7043B1A68C2401A60F2E7C04602
:08118000641400209814002003
:10118800054B1A68111F1268086802400A601A683D
:0C119800043A1A607047C046641400203E
:1011A400054B1A68111F1268086802430A601A681E
:0C11B400043A1A607047C0466414002022
:1011C000054B1A68111F1268086842400A601A68C5
:0C11D000043A1A607047C0466414002006
:1011DC00024B1A681368DB431360704764140020D9
:1011EC00024B1A6813685B4213607047641400204A
:1011FC00054B1A68111F1268086842430A601A6886
:0C120C00043A1A607047C04664140020C9
:1012180010B50B4B1C682168002909D0043C2068D4
:1012280005F02AFF2060064A1368043B136010BDCE
:10123800044A80231B0111680B431360F7E7C0467B
:0812480064140020981400203A
:1012500010B50B4B1C68216800290AD0221F1068AA
:10126000083C23685843064B1C6005F009FF2060CA
:1012700010BD044A80231B0111680B431360F7E77C
:08128000641400209814002002
:1012880010B50B4B1C682168002909D0043C206864
:1012980005F024FF2160064A1368043B136010BD63
:1012A800044A80231B0111680B431360F7E7C0460B
:0812B8006414002098140020CA
:1012C00070B50D4B1C682568002D0ED0043C2668B7
:1012D0002900300005F006FF2160074B1C6829003B
:1012E000300005F0CDFE206070BD044A80231B0154
:1012F00011680B431360F7E7641400209814002072
:10130000034A1368191D1160024A12685A60704737
:081310006414002068140020A1
:10131800064A1368191F1B6808681B1A584243417C
:101328000B601368043B13607047C04664140020C8
:10133800064A1368191F1B6808681B1A581E834140
:101348000B601368043B13607047C04664140020A8
:10135800034B1A6811684B424B4113607047C046F3
:0413680064140020E9
:10136C00074B1A68131F012112681868904200DCA1
:10137C0000211960024A1368043B13607047C04691
:04138C0064140020C5
:1013900030B5074B1A68111F10680A68D217C40FBE
:1013A0000D68854262410A601A68043A1A6030BDCD
:0413B00064140020A1
:1013B400074B1A68131F012112681868904200DB5A
:1013C40000211960024A1368043B13607047C04649
:0413D400641400207D
:1013D800064A1368191F1B68086884469C459B4188
:1013E8005B420B601368043B136070476414002071
:1013F80030B5074B1A68111F08681468C20FE51743
:1014080084426A410A601A68043A1A6030BDC046CC
:041418006414002038
:10141C00044B0A221A60044B1B68002B01D1034BAE
:10142C001A607047501400209C1400207C1400207B
:10143C00044B10221A60044B1B68002B01D1034B88
:10144C001A607047501400209C1400207C1400205B
:10145C000F4B1B68012B05D00E4A402311680B4320
:10146C00136070470C4B19680A1D1A600B4B1B68F4
:10147C000B4A1268934203D005D2D31A4B60F0E7A3
:10148C0000234B60EDE79B1AC4334B60E9E7C04681
:10149C00081500209814002064140020FC1400206F
:0414AC000015002007
:1014B00006490A681368043A0A60002B05D00449FB
:1014C000044A0A60013B002BFBD1704764140020E2
:0814D00000300040AAAA000050
:1014D80004490B6864221868424303480260043BCD
:0C14E8000B6070476414002054140020B6
:1014F40010B5054B1C68221D1A60044B1868642142
:1015040005F0DAFD606010BD64140020541400205E
:1015140030B5094B1B68013B08495B181B041C0CC4
:10152400074802681B0E15684B5513689C466144B6
:101534004C70043A026030BDA81400201002002050
:04154400641400200B
:10154800044B1A68111D1960034B1B68043B1B6888
:0C15580053607047641400206C140020E5
:10156400024B1B681A68024B1A6070476C14002007
:0415740090140020AF
:10157800064B1B681A68002A04D1054A12681168CC
:10158800044A1160043B014A136070476414002048
:081598006C14002090140020E7
:1015A000154B1B68154A19681160154A934218D9E2
:1015B000144A1268022A07D0043B0F4A1360124AE9
:1015C0001368013B136070470F4A11680F4A126895
:1015D0009142F1D10D4A002111600A4A0331116094
:1015E000EAE7064B00221A60064B1B68022BEAD181
:1015F000044B03321A60E6E76C14002090140020BC
:10160000F8120020FC01002084140020B4140020F3
:10161000054B00221A605A609A6018000C3003498A
:101620000860DA607047C0465C1300206414002034
:0C163000014B03221A607047FC010020EF
:0C163C00014B01221A607047FC010020E5
:0C164800014B00221A607047FC010020DA
:1016540030B50D4B1C68221D1A600C490B685A1CCE
:101664000A60587800069A1C0A609A7812040243A9
:10167400D81C0860D87800021D1D0D601B79134327
:101684000343636030BDC0466414002090140020FE
:10169400054A1368191D116004490A68501C086042
:1016A40052785A607047C046641400209014002099
:1016B400074B19680A1D1A60064A1368581C106003
:1016C4005A781201044B9B189B684B607047C046C4
:0C16D40064140020901400201008002076
:1016E000074B1A68511C19600648036851780901B4
:1016F000054A521819689160043B03607047C04660
:0C17000090140020641400201008002049
:10170C00074B1A68511C196051780902901C18601B
:10171C0092781143802292050A431A607047C046A2
:04172C0090140020F5
:1017300010B5094B1868021D1A6008490B685A1C3D
:101740000A605A7812029C1C0C609B781A43802312
:101750009B051343436010BD6C14002090140020BF
:10176000084B094A1A60094B1A68511C19605178D4
:101770000902901C186092781143802292050A4356
:101780001A60704700300040AAAA000090140020A0
:1017900010B5094B1B681A68023A80239B05134356
:1017A0001A78752A03D1013B044A136010BD034A1D
:1017B0001360FFF7D5FFF9E76C14002090140020A8
:1017C00010B50A4B1B681B68002B0CD0084A136825
:1017D000043B1360074A136803331360034A13681A
:1017E000043B136010BDFFF7BBFFF7E76414002054
:0817F0006C140020901400208D
:1017F80010B50A4B1B681B68002B0CD1084A1368EC
:10180800043B1360074A136803331360034A1368E1
:10181800043B136010BDFFF79FFFF7E76414002037
:081828006C1400209014002054
:1018300010B5104B1A681100103119600E490B6871
:10184000180008380068D060181F00689060186899
:1018500050600C3B0B6009480368591C01605978C3
:1018600009029C1C04609B78194380239B050B4351
:10187000136110BD6C14002064140020901400202B
:1018800010B5254B1B681A1F126819000839086823
:101890000C3B19685318214A214C146000291DDBA8
:1018A000984212DD1C4A1268043A13601D4B1A68F4
:1018B000511C196051780902901C186092781143EC
:1018C000802292050A431A6010BD134A1368103B28
:1018D0001360144A136803331360F5E7984212DA71
:1018E0000D4A1268043A13600E4B1A68511C1960B5
:1018F00051780902901C1860927811438022920559
:101900000A431A60E0E7044A1368103B1360054A73
:10191000136803331360D7E76C14002000300040D5
:08192000AAAA000090140020A7
:10192800024A1368043B13607047C0466C140020D9
:10193800024A1368103B13607047C0466C140020BD
:1019480010B5044C23681878FEF75CFC2368043B48
:08195800236010BD641400209F
:1019600000B583B06A46094B03CB03C2084B1B6822
:10197000002B01D003B000BD684605F0E6F8044B2B
:1019800001221A60034B00221A60F3E74C6300083F
:08199000FC01002048140020B6
:1019980010B5114B1B68002B12D0104B1B78002B75
:1019A8000ED00F4B1B68002B15D00E4A1368191D5B
:1019B80011600D4A12785A60094B00221A600AE039
:1019C800FFF700FA0028FBD0064B1A68111D1960B2
:1019D800FF231840506010BDFC0100202B1500208B
:0C19E8004C140020641400202A1500207C
:1019F40010B50E4B1B68102B08D00D4B1B681868D4
:101A0400E0231B06C2180B4B9A420CD8084B1B68E8
:101A1400186805F027FB2020FEF7F6FB044A13683C
:101A2400043B136010BDFEF7BFFFF4E75014002021
:081A340064140020FF0B0630D2
:101A3C0010B5064C2368186805F010FB2020FEF743
:101A4C00DFFB2368043B236010BDC04664140020F8
:101A5C00F0B587B003AA2A4B13CB13C2294B1A68D3
:101A6C0001929A8801AB9A805B20FEF7C9FB264B4A
:101A7C001B68264A0C3293420DD0244A0C329342F6
:101A8C000DD3224A0C32934216D9204C1034042523
:101A9C001E4F160024E001A805F051F80CE003A835
:101AAC0005F04DF8194B00221A605A609A60180024
:101ABC000C3015490860DA605D20FEF7A1FB202090
:101ACC00FEF79EFB07B0F0BD206805F0C7FA20209A
:101ADC00FEF796FB01350C4B1B680434B342EBD973
:101AEC00DB1B9B10AB42E7D32020FEF789FB084B96
:101AFC001B68102BE8D02068FEF752FFE7E7C046C2
:101B0C001C6B0008286B0008641400205C13002078
:041B1C005014002041
:101B2000F0B5D6464F464646C0B584B001AA394BFB
:101B300003CB03C21B7813702020FEF767FB364BE4
:101B40001B68002B5BD0354D00270026C0231B05EA
:101B50009946334B9A46304B984616E02020FEF7C4
:101B600055FB14E06B684A46134221D12020FEF752
:101B70004DFB2020FEF74AFB01360137052F34D8F4
:101B8000103543461B68B34237D9092EE6D93000D9
:101B9000FEF70CFF3A20FEF739FB2C00083C2078BA
:101BA0000028DFD0FEF732FB0134AC42F7D1D9E791
:101BB00001A804F0CAFF53461B68102B11D02868F7
:101BC000FEF7F4FE2020FEF721FB4020FEF71EFB6F
:101BD0002804000C05F048FA2920FEF717FB02370D
:101BE000C4E7286805F040FAECE70D20FEF70EFB8D
:101BF0002020FEF70BFB0027C2E7002F05D104B021
:101C0000E0BCBA46B146A846F0BD0D20FEF7FEFA8C
:101C1000F5E7C046646D0008801400201808002015
:041C2000501400203C
:101C240010B5044C2368186805F03BF82368043B9E
:081C3400236010BD64140020C0
:101C3C0010B5074B1B68002B04D1064A1368043BF4
:101C4C00136010BD034B1B681878FEF7CDFAF4E750
:081C5C000815002064140020AB
:101C6400F0B5C64600B5114A13681F68043B1360FB
:101C7400002F13D00125ED1BAD003C000C4E904607
:101C840003E0013C0435002C08D03368002BF8D065
:101C940043461B68585DFEF7ABFAF2E7034BBF00FF
:101CA4001A68D71B1F6080BCB846F0BD64140020BE
:041CB40008150020EF
:101CB800F0B5C64600B582B06846214B020012CB8B
:101CC80012C204F03EFF0D20FEF79CFA1D4DFC23C6
:101CD8009B009846A8440026012723E0FEF792FAC5
:101CE8000134285D0028F9D1062C05D82020FEF7FC
:101CF80089FA0134072CF9D12320FEF783FA38003A
:101D080004F047FF2020FEF77DFA2020FEF77AFA3C
:101D18002020FEF777FA01370136052E07D008355F
:101D2800A84509D02020FEF76DFA0024D9E70D2038
:101D3800FEF768FA0026F2E702B080BCB846F0BDAC
:081D4800546300083066000836
:101D500070B5FFF73BF8041E00D1D8E0C0B2704B5D
:101D60001B68002B08D06F4B1B78002B04D06E4BE8
:101D700018706E4B01221A600A2800D1C4E00228B4
:101D800000D8C3E0674B1B78002B08D109281FD06F
:101D9000674A12683F2A02D9202800D19EE02828ED
:101DA00018D02F2840D01B2868D10024002B00D148
:101DB000ADE00E38FEF72AFA5D4B1A685D4B202124
:101DC00099549B18002159705B4B1A6002349EE0B5
:101DD0001730DDE7594B1C68002C01D0002496E039
:101DE000FEF714FAFEF7F2FF0028FBD0C0B220285D
:101DF0000BD04F490B684F4A2825D554D218507044
:101E000002330B60FEF702FA81E0494B1B68013395
:101E10004A4A13601838FEF7F9F92020FEF7F6F960
:101E20000820FEF7F3F972E0444B1C68002C01D047
:101E300000246CE0FEF7EAF9FEF7C8FF0028FBD0AB
:101E4000C0B22F280BD03A490B683A4A2F25D554F7
:101E5000D218507002330B60FEF7D8F957E0344BBC
:101E60001B680133354A13602738FEF7CFF920206D
:101E7000FEF7CCF90820FEF7C9F948E0092848D058
:101E8000122848D0082817D12C4B1D680024002D9B
:101E90003DD1274B1C68002C39D0013C1C60254BE0
:101EA00020221A55FEF7B2F92020FEF7AFF90820DC
:101EB000FEF7ACF92C002AE00D2817D11C4B1B684B
:101EC000002B0BD11A4B1A681A4B202199549B18DE
:101ED00000215970184B1A60012418E0174B1B6839
:101EE000012BEFD00D20FEF791F9EBE7134B1C68A7
:101EF000002C12D10E4D0F4B2A689854FEF786F92C
:101F00002B6801332B6002E0002400E00024200055
:101F100070BD0324FBE70424F9E70024F7E7C0467B
:101F2000FC0100202B1500202A1500204C14002055
:101F3000401400209412002044140020A01400201B
:101F400010B50023054A1360054A1360054A136063
:101F5000FFF7FEFE0028FBD010BDC0464014002055
:081F600044140020A01400202D
:101F680010B5154B1968154B5A5C202A09D14B1C22
:101F78001248013819000133C25C202AFAD00E4BEE
:101F880019600023002A10D00C4840180C4CC25C81
:101F9800202A03D01A5501330F2BF8D1084A002004
:101FA800D0545B18074A136010BD054B00221A7005
:101FB800044B1960F8E7C04638140020941200203A
:081FC800C013002040140020AA
:101FD000F0B5DE46474680B587B00E0002AA002461
:101FE00005E0002B1BD001340132102C08D0035D1A
:101FF0001370190061391929F3D8203B1370F2E7E7
:10200000002302AAD37313782D2B0ED1254B002267
:102010001A6001239B460127012C0FD82CE00023D6
:1020200002AAD37313782D2B2CD01E4B00221A60DA
:1020300000239B4600270120002C2DD0194B1D6842
:10204000B84602AB9C46E04400230193434618780F
:10205000310004F034FE431C18D075432D180137AD
:1020600001239C46E0440193A742EFD30D4B1D6032
:1020700001205B46002B0FD00A4A13685B421360B5
:10208000012009E00020012CC0D105E0019B002BBC
:1020900001D0044B1D60002007B0C0BCBB46B04659
:0820A000F0BDC0463C14002015
:1020A80010B5344B187800285AD000233149013331
:1020B8005A5C002AFBD12D280FD0302829D12D4A6F
:1020C800527820218A43582A11D02B4A11681029A6
:1020D8003AD1082B48D900204BE0012B3AD0264AA8
:1020E800116810292AD00B2B3ED9002041E0214A43
:1020F80092782D2A09D00A2B2ED81E48102102309A
:10210800FFF762FF431E984133E00B2BF5D90020FF
:102118002FE02528D9D1174A52782D2A09D00B2B20
:102128001CD814480A210130FFF74EFF431E98417E
:102138001FE00C2BF5D900201BE000232D28C8D167
:10214800092B11D9002014E02D28CCD000200A2B0F
:102158000FD809E000200CE000200AE0002008E089
:10216800054B19681029E8D00248FFF72DFF431ED8
:0C217800984110BDC0130020501400203E
:10218400F0B51A4C00251A4E0021635C8A5D1800D4
:10219400613819280DD8203BDBB2100061381928AA
:1021A40011D8203AD2B2934219D101310829ECD185
:1021B40015E01000613819280DD918002038471E81
:1021C400B84140420340934209D1002AEDD1094B62
:1021D4001D600120F0BD203AD2B2202BE3D101359D
:1021E40008347F2DD0D10020F4E7C04628660008CB
:0821F400C0130020701400204C
:1021FC0070B51A4B1B78002B29D0194A00231E00EE
:10220C00013310321100103909780029F7D1731CF1
:10221C001FD03301114C1C19124D16E08B4211D1F9
:10222C0000290BD00132082A0CD0A15C535D180098
:10223C0061381928F2D8203BDBB2EFE70A4B1E605D
:10224C00012070BD103C013E05D30022EDE70020BB
:10225C00F7E70020F5E70020F3E7C0461008002060
:0C226C0020080020C01300207014002087
:1022780010B50F4B1A680F4B1A60FFF771FEFFF786
:10228800B9FF002805D00C4B1B6801330B4A1360BB
:1022980010BD0B4B1B78302B05D00A4A212311683F
:1022A8000B431360F4E7054B00221A60F0E7C046C1
:1022B800401400203814002070140020B8140020A6
:0822C800C0130020981400204F
:1022D000074A13680749C85401331360064A9342FA
:1022E00004D9064A202311680B4313607047C04687
:1022F000A814002010020020FE0500009814002001
:1023000010B5144B18688200134BD3581A030AD423
:10231000124A1268002A13D19B030BD48000104B81
:10232000C358984705E00F4A80239B0011680B4370
:10233000136010BD0B4A082311680B431360F8E7C4
:10234000DB0304D58000064BC3589847F1E7FFF73D
:10235000BFFFEEE7701400202C6400089C140020DE
:08236000000000209814002089
:1023680070B594B00CA9414B0A0013CB13C213CB20
:1023780013C203CB03C205A93D4B0A0013CB13C2FA
:1023880013CB13C21B7813706A463A4B13CB13C294
:1023980011001A680A601B790B71374B1B68522BA6
:1023A80009D95224354E344DA05DFDF72BFF013479
:1023B8002B68A342F8D85223314A1360314A0021CE
:1023C8001160314A13602E4D304E03E02C4B1A68D1
:1023D8002D4B1A60284C2B682268934234D2FFF7A1
:1023E800BFFD3378002BF6D0FFF75AFE00280BD03C
:1023F800274B1A68274B1A60274B1B78002BE5D010
:10240800264B01221A60E1E7FFF7B8FE002811D039
:10241800234B1B689B00234A9B585B0321D5FFF77E
:102428006BFF214B1B68002B08D1154B1A68164B04
:102438001A60CFE70CA804F084FB05E01A4B0022D1
:102448001A60684604F07DFB0D20FDF7DBFE522381
:10245800094A13600A4A13600A4B00221A6014B032
:1024680070BD05A804F06DFBEEE7C0467C6D000862
:102478009C6D0008B86D00084414002094120020D8
:1024880040140020A014002038140020C01300209D
:102498003C140020AC1400202B150020B0140020A0
:0C24A800701400202C6400089814002020
:1024B40070B56F20FFF70AFF0C4D2C68FF20FFF763
:1024C40005FFFF20FFF702FF2B68013B084A9B181A
:1024D4001B04180C074909681B0E0D6853550B683B
:1024E4009C46624450700C6070BDC046A814002025
:0824F400100200206414002016
:1024FC0010B57020FFF7E6FE064A1368191D11602F
:10250C00054A12685A60FF20FFF7DCFEFF20FFF738
:0C251C00D9FE10BD64140020A81400209B
:1025280010B57420FFF7D0FE064A1368191D116014
:10253800054A12685A60FF20FFF7C6FEFF20FFF722
:0C254800C3FE10BD64140020A814002085
:10255400F8B57520FFF7BAFE104E33681D680135D3
:102564000F4C2D19280AFF273840FFF7AFFE38001B
:102574002840FFF7ABFE0B4B1B68013B1B1932686D
:10258400190A106821541268A41863707720FFF7A1
:102594009DFE3368043B3360F8BDC04664140020DC
:0825A40010020020A814002021
:1025AC0010B51F4B1B68002B17D11E4B1B681E4A06
:1025BC00196811601D4A93422ED91D4A1268022ACD
:1025CC001DD0043B174A13601A4A1368013B136071
:1025DC00194B1A68194B1A6010BD6420FFF772FE74
:1025EC0000220F4B1A6016490B6801330B601B015C
:1025FC0014495A54144B1A68144B1A60E8E70D4AE4
:10260C001168134A12689142DBD1114A0021116002
:10261C00074A03311160D4E7034B00221A60D7E755
:10262C009C1400206C14002090140020F812002040
:10263C00FC010020841400207C1400205014002085
:10264C008014002010080020A8140020A4140020DE
:04265C00B414002092
:1026600070B5324B1B68002B27D1314B1B681C788F
:1026700023005F3B022B16D97D20FDF7C7FD2020EC
:10268000FDF7C4FDFFF7EAF92500703D072D15D9C8
:10269000743C012C1CD9032D0FD8264B1B681888BD
:1026A00004F0ACFC09E0244B186801300005000D73
:1026B00004F0A4FC2920FDF7A9FD70BD2020FDF742
:1026C000A5FD5220FDF7A2FD3A20FDF79FFDDFE7B3
:1026D000184B1A68194BD31A082BEED90C3A1088EC
:1026E00004F08CFC2020FDF791FD2020FDF78EFDED
:1026F000104C2368083B188804F080FC2020FDF76C
:1027000085FD6920FDF782FD2368043B188804F0ED
:1027100075FC2020FDF77AFD7820FDF777FD236812
:102720001888013004F06AFCC7E7C04698140020FE
:102730008C1400206C14002090140020F81200204B
:10274000104B1B68002B0BD00F4B18680F4B1B68EE
:10275000984205D001D2181A13E0C01AC43010E014
:102760000B4B186800280BD10A4B1B680A4A1268E9
:10277000934206D0D01A934203D3981AC43000E093
:10278000002070472C140020CC140020D01400200E
:0C27900008150020FC140020001500209B
:10279C0010B5094B1C68221D1A60084B1B68002BD6
:1027AC0006D0074B1B78002B02D0064B186801E0B3
:1027BC00FFF7C0FF606010BD64140020FC01002016
:0827CC002B1500204C14002025
:1027D40010B50B4B1C6800230A4909190A48CA5C46
:1027E400222A03D01A5401334E2BF8D1064A22214F
:1027F400D15401330021D154E318044A136010BDAD
:102804003814002094120020C0130020401400202B
:102814001A4B1B185A781300613B192B03D8203A22
:102824001300373B05E02F2A1BD91300303B092B3B
:10283400F6D80F2B18D8114A101882781100613974
:10284400192907D8203A373A11000F2912D818014C
:10285400401870472F2A0AD9110030390929F4D9B0
:10286400F1E701204042F4E701204042F1E7012072
:102874004042EEE701204042EBE7C046C01300208F
:10288400F0B5C64600B50700404B1B680133404A0B
:102894001360FFF79DFF002600243E4A03E0013643
:1028A4000134502C10D0A35C5C2BF8D0222BF7D130
:1028B400384B00221A55384B1D68002D0CD1354C6D
:1028C400364B98461E003BE0354A022311680B4301
:1028D400136080BCB846F0BD012F0ED06620FFF710
:1028E400F5FC304A13687600A41B2F49CC540133FD
:1028F40013600024274D2E0009E06520FFF7E6FC55
:10290400EFE7FFF7E3FC0134335D002BE1D0285DF2
:102914005C28F6D12000FFF77BFF431C03D003346F
:10292400FFF7D4FCF0E71E4A022311680B4313603F
:10293400CFE7FDF769FC0135164B5B5D002BC8D072
:10294400605D5C2807D0012FF3D03368002BF2D0F0
:10295400FDF74EFCEFE72800FFF75AFF431C0AD0AF
:102964000335012F0DD043461B68002BE4D0C0B2C1
:10297400FDF73EFCE0E70A4A022311680B431360AB
:10298400A7E7C0B2FDF740FCD6E7C04640140020DC
:1029940038140020C01300209C14002008150020C7
:0C29A40098140020A8140020100200204D
:1029B00010B5154B1B68022B17D0144B1868002854
:1029C00017D0134B1B780020002B12D0FFF7B8FE56
:1029D00000280ED0FFF7BCF901280BD002280CD03C
:1029E0000C4B1868431E984103E0074B00221A6005
:1029F000012010BDFFF7B8FCF2E7064A80235B0018
:102A000011680B431360EBE748140020FC01002021
:082A10002B1500209814002092
:102A180010B50D4B1B68012B05D00C4A40231168DB
:102A28000B43136010BDFEF7A1F9002804D1FFF78E
:102A3800BBFF0028F7D0F5E7054B1A68111D196090
:102A4800FF2318405060EDE7081500209814002077
:042A580064140020E2
:102A5C0010B5094A1368094918680860043B1360EB
:102A6C000C002368002B05D0FDF716FDFFF79AFF2D
:102A7C000028F6D010BDC046641400208814002035
:102A8C0010B5044B1A68642311684B431360FFF7AD
:082A9C00DFFF10BD64140020EF
:102AA40070B5394B1B6880225202934231D3364BA6
:102AB400364A1A60364B1B88DB0711D4344B00228C
:102AC4001A821A803349CA6902200243CA61324A0F
:102AD4001A83FA22D200DA621A8801210A431A8080
:102AE400294B1B68013B9BB2294A13852B4B1B685E
:102AF400002B3DDB264A138C01210B431384284B06
:102B04001B68002B39DB224A138C10210B431384DE
:102B14002DE0002BCED11E4A13880125AB43138030
:102B2400012464421D4B1C609023DB0518681D4E74
:102B340030401860D9683140D960D8688021890153
:102B44000143D960118CA943118415490C6018689C
:102B5400154C20401860D9682140D960D86880217C
:102B640009020143D960138C10218B43138470BD77
:102B7400138C01218B431384C1E7054A138C102164
:102B84008B431384F3E7C04694140020FFFF000036
:102B9400000400400010024060600000781400202F
:0C2BA40074140020FFCFFFFFFF3FFFFF75
:102BB0009022D205136827490B401360264A138CD4
:102BC00001218B431384254B1B68002B24DB9021B0
:102BD000C905CA681F480240CA60002B24D0FA22E7
:102BE000D20093422ADA9023DB05196880229201F1
:102BF0000A431A601A6A1A490A401A62196A80223C
:102C000052040A431A62144B1A8C01210A431A8493
:102C1000124A12685A6370479022D205D168802305
:102C20009B010B43D360F6E70B0009688022520139
:102C30000A431A608022D2039A61ECE7074B1A60BC
:102C40009023DB051968802252010A431A60402252
:102C50009A61E0E7FFCFFFFF0004004078140020F6
:042C6000FFFFFFF083
:102C64009022D205136827490B401360264A138C1F
:102C740010218B431384254B1B68002B24DB9021EC
:102C8400C905CA681F480240CA60002B24D0FA2232
:102C9400D20093422ADA9023DB05196880221202BB
:102CA4000A431A601A6A120112091A62196A802206
:102CB40052050A431A62144B1A8C10210A431A84CF
:102CC400124A12689A6370479022D205D168802311
:102CD4001B020B43D360F6E70B0009688022D20184
:102CE4000A431A60802212049A61ECE7074B1A60C7
:102CF4009023DB0519688022D2010A431A608022DE
:102D04009A61E0E7FF3FFFFF0004004074140020D5
:102D1400114A13681868043B136018280BD9030080
:102D2400A03B182B05D90D4A8023DB0011680B4307
:102D340013601F2318400300083B042B04D9042309
:102D440002009A43122A05D1044A8023DB00116849
:102D54000B4313607047C04664140020981400208D
:102D640010B5FFF7D5FF104B1B68002B0FD10F28B0
:102D74000ED89023DB051B8A0122824013400B49A5
:102D84000A68101D0860002B0AD00123536010BD8F
:102D9400074B1B8A0F2210400E3A82401340EEE785
:102DA40000235360F3E7C046981400206414002005
:042DB40000040048CF
:102DB80006280FD007281AD10D4B1B68013316D0EF
:102DC8000C4A138C10218B431384094B0122524265
:102DD8001A600CE0084B1B68013308D0054A138CB5
:102DE80001218B431384044B012252421A6070471D
:0C2DF80074140020000400407814002037
:102E040070B5FFF785FF0400174B1B68002B14D126
:102E14000F2813D9400003228240144BD9689143F0
:102E2400D9601968914319601D680122110081401D
:102E340029431960103CA2409A6170BDFFF7BAFFA4
:102E44006000032282409023DB05D9689143D96056
:102E54001968914319601D680122110081402943BA
:102E64001960A2409A61E8E7981400200004004821
:102E740070B5FFF74DFF0400174B1B68002B13D1EF
:102E84000F2812D9400003228240144BD968914381
:102E9400D9601968914319601D68012211008140AD
:102EA40029431960A2409A6170BDFFF783FF600057
:102EB400032282409023DB05D9689143D9601968C5
:102EC400914319601D680122110081402943196052
:102ED4001034A2409A61E7E79814002000040048E7
:102EE40010B5FFF715FF0400144B1B68002B11D11C
:102EF4000F2810D9103C64000322A240104B19681B
:102F040091431960D9689143D960D9680122A240DC
:102F14000A43DA6010BDFFF74DFF64000322A240AC
:102F24009023DB05196891431960D9689143D960EE
:102F3400D9680122A2400A43DA60EBE79814002022
:042F4400000400483D
:102F480010B5FFF7E3FE0400144B1B68002B10D1EB
:102F58000F280FD944000322A240114B196891434E
:102F68001960D9689143D960D9680222A2400A43FE
:102F7800DA6010BDFFF71CFF64000322A240902313
:102F8800DB05196891431960D9689143D960D968FC
:102F98000222A2400A43DA60EBE7C04698140020F8
:042FA80000040048D9
:102FAC0010B5FFF7B1FE04000F4B1B68002B0BD1C3
:102FBC000F280AD944000322A2400C4B19689143F4
:102FCC001960D9689143D96010BDFFF7EFFE64001A
:102FDC000322A2409023DB05196891431960D9683C
:102FEC009143D960F0E7C0469814002000040048D3
:102FFC0010B5144BDA6814490A40DA6099698022DA
:10300C0092000A439A61FDF761F8FDF75FF8FDF74E
:10301C005DF8FDF75BF80D4B802212061A61002259
:10302C00DA600B490A6004325A619A6801210A433A
:10303C009A60190001220B681A42FCD0FDF746F881
:10304C0010BDC04600100240FFFDFFFF00240140F0
:04305C000827014000
:103060000C4B1A6801210A431A609A6801310A431D
:103070009A60190001228B681A42FCD1064B9A69AA
:1030800006490A409A61D968802292000A43DA60B0
:103090007047C0460024014000100240FFFDFFFFC2
:1030A000F0B589B004AA5C4B13CB13C21B88138004
:1030B0006A465A4B13CB13C21B781370584B1B68CC
:1030C0001C68621C18D0072C03D92300A03B072BD7
:1030D0001BD8544B9B699B051ED5534B534A1A6012
:1030E0000F232340590003228A40072B00D98BE08D
:1030F00099004F4841588F46043B494A1360FFF7F7
:10310000AFFF684603F021FD35E04A4A8023DB002B
:1031100011680B4313602EE0FFF770FF04A803F063
:1031200014FDDAE79021C905086810430860C868F3
:103130009043C86001229A4013003B4A93620426E0
:10314000002714000425A3682B43A36023681D42B5
:10315000FCD0236CFF18FCF7BFFF013E002EF2D11C
:103160002F4B1B68BA081A60BB0704D52C4B1A6892
:1031700013680133136009B0F0BD9021C9050868D8
:1031800010430860C8689043C860D3E79021C90520
:10319000086810430860C8689043C860CAE7902177
:1031A000C905086810430860C8689043C860C1E753
:1031B00021490968013108D02048018C0124A1432C
:1031C00001841D490120404208609021C90508681A
:1031D00010430860C8689043C860ABE718490968A5
:1031E000013108D01548018C1024A14301841449F1
:1031F0000120404208609021C9050868104308601A
:10320000C8689043C86095E70A4A8023DB001168CC
:103210000B431360AFE7C046D86D0008E86D0008A7
:10322000641400200010024000240140FF07000049
:103230005C6300089814002078140020000400400B
:0432400074140020E2
:103244001A4B1B68032B25D8194B1B68043B1C2BFA
:1032540020D880235B02174A12689A421AD2164B6E
:103264001A6816490A401A6019688822D2000A436B
:103274001A60DA6812490A40DA60D968802292003A
:103284000A43DA60094B1B68012B0AD90A4B08224E
:103294009A6105E00B4A8023DB0011680B4313603D
:1032A4007047054B802212039A61F9E758140020F5
:1032B400601400205C140020000400483FF0FFFF6D
:0832C400FFFCFFFF981400203D
:1032CC0010B50A4A13680A4918680860191F11607A
:1032DC00086808490860190008391160086806492F
:1032EC0008600C3B1360FFF7A7FF10BD64140020AF
:0C32FC005C140020601400205814002016
:10330800F8B5DE4657464E464546E0B5B54B1B6810
:10331800A822D2001340013AFF3A93421BD1B24B84
:103328001B681C68B14B1A68B14B186800286DD12E
:10333800AC4B802109039961AE4B1B68002B0DD162
:103348000125A84880218903884620218C468027AA
:103358003F03082644E0FFF771FFE0E701239B469F
:10336800A04D80239B039A462023994680231B0364
:103378009846A04B9C46A0491F001EE05346AB61EF
:103388004346AB6163461B68002B04D09B4E3160FB
:10339800013B002BFBD140002B8A1B095E463340C2
:1033A80018430823AB613B68002B04D0934E31606F
:1033B800013B002BFBD1002A1BD0013A5B4693400E
:1033C8001C42DBD04B46AB61DAE74146816187613D
:1033D8005900038A1B092B400B438661002A07D03A
:1033E800013A290091400C42EFD061468161EEE735
:1033F80018007C4B802212039A617B4B1B68186073
:10340800F0BCBB46B246A946A046F8BD012814D078
:10341800022875D0734B08219961764B18680028EB
:1034280000D0CDE001256F4980239B0398462023D7
:103438009C4680273F03082614E16A4B8021090334
:1034480099616C4B186800280AD1012565498023C9
:103458009B03984620239C4608278026360342E093
:10346800002001239B465F4D80239B039A4620231F
:103478009946183B98465F4B9C465F491F001FE0E2
:103488005346AB614346AB6163461B68002B04D0CF
:103498005A4E3160013B002BFBD140002B8A1B099F
:1034A8005E463340184380231B03AB613B68002B07
:1034B80004D0524E3160013B002BFBD1002A1AD0B8
:1034C800013A5B4693401C42DAD04B46AB61D9E7E0
:1034D80043468B618F6140000B8A1B092B401843C0
:1034E8008E61002A07D0013A2B0093401C42EFD08E
:1034F80063468B61EEE73B4B802212039A617CE7BF
:10350800384B082199613B4B186800280AD10125DE
:10351800344B80218903884620218C460827802641
:10352800360341E0002001239B462E4D80239B0358
:103538009A4620239946183B98462E4B9C462E497E
:103548001F001FE05346AB614346AB6163461B68EF
:10355800002B04D0294E3160013B002BFBD14000E9
:103568002B8A1B095E463340184380231B03AB613B
:103578003B68002B04D0214E3160013B002BFBD16E
:10358800002A19D0013A5B4693401C42DAD04B46D8
:10359800AB61D9E7414699619F614000198A29408A
:1035A80008439E61002A07D0013A290091400C4245
:1035B800F0D061469961EFE70A4B08229A611CE74F
:1035C800002001239B46074D80239B039A46202316
:1035D800994680231B039846064B9C4606491F00C4
:1035E8002DE0C04600040048641400206014002048
:1035F800581400205C140020AAAA000000300040E3
:103608005346AB614346AB6163461B68002B04D04D
:103618001A4E3160013B002BFBD140002B8A1B095D
:103628005E46334018430823AB613B68002B04D047
:10363800124E3160013B002BFBD1002A1AD0013A0F
:103648005B4693401C42DBD04B46AB61DAE743460E
:103658008B618F6140000B8A1B092B4018438E61D8
:10366800002A07D0013A2B0093401C42EFD0634652
:103678008B61EEE7024B08229A61BEE600300040FB
:0436880000040048F2
:10368C0010B5074A1368191D1160064A12685A6072
:10369C00FF20FEF717FEFF20FEF714FE10BDC046FC
:0836AC0064140020A8140020A2
:1036B400F8B5104E33681D6801350F4C2D19280AD2
:1036C400FF273840FEF702FE38002840FEF7FEFDD3
:1036D4000A4B1B68013B1B193268190A10682154F4
:1036E4001268A41863707620FEF7F0FD3368043B7B
:1036F4003360F8BD6414002010020020A8140020D8
:1037040070B57E280DD8C0000E4D441908352D180B
:103714002078002804D0FCF777FD0134AC42F7D1BF
:1037240070BD7F2528400001074D441908352D1828
:1037340020780028F4D0FCF767FD0134AC42F7D1BF
:0C374400EEE7C0462866000810080020D0
:1037500070B50001064D441908352D182078002851
:1037600004D0FCF753FD0134AC42F7D170BDC04624
:04377000100800201D
:10377400F0B5C64600B582B0A34B1A6800929B8888
:103784006A469380A14B1D68002D03D002B080BC13
:10379400B846F0BD9E4B1B689E4A13601B78984642
:1037A4001F009D4B1B685E00F6180D20FCF72CFDD6
:1037B400002E06D02C002020FCF726FD0134A64262
:1037C400F9D1944B188803F017FC2020FCF71CFD5A
:1037D400404603F011FC2020FCF716FD7F2F1AD879
:1037E4004046FFF78DFF6B2F53D06C2F57D06D2FB2
:1037F40000D182E06E2F00D187E06F2F56D0712F59
:1038040000D18AE0722F00D18DE0FD224346733B44
:1038140013424BD059E02D20FCF7F6FC3E20FCF778
:10382400F3FC2020FCF7F0FC4046FFF769FF784BDF
:103834001B685B787F241C40692F00D19EE06A2FAF
:1038440000D1A5E0642F00D1B7E0744C032D00D162
:10385400C7E02368022B00D8C3E0FCF721FEFEF783
:103864006DFF0028F2D0FEF771FA0500012800D19F
:10387400ADE0022800D1ADE00428E7D1664B1B6817
:10388400002B00D1ADE0664A1360644B02221A603B
:10389400DCE7644B1B681B68002B07D0C7E7614B50
:1038A4001B68191F1A680B689A42C0D0684603F057
:1038B4004AF9574B1B68587800029B78184301302B
:1038C40003F09AFB2920FCF79FFC682F35D1504B5D
:1038D4001B685C782820FCF797FC534B1B68102B63
:1038E40027D02000FDF760F82920FCF78DFC484B19
:1038F4001B685B787F241C40A1E74A4B1B681A1F96
:1039040012681B689A42D1D291E7464B1B681A1F72
:1039140012681B689A42C9D989E7424B1B681B6825
:10392400002BC3D083E73F4B1B681B68002BBDD122
:103934007DE7200003F060FBD6E7672F00D076E731
:10394400334B1A6893781B04517809060B43117999
:103954000B43D47824021C432820FCF755FC324B3B
:103964001B68102B06D02000FDF71EF82920FCF759
:103974004BFC67E7200003F03FFBF7E72820FCF748
:1039840043FC2000FFF7E2FE2920FCF73DFC5CE746
:103994002820FCF739FC2000FFF7D8FE4020FCF774
:1039A40033FC20010830214C00190004000C03F002
:1039B40059FB2920FCF728FC47E72020FCF724FCCE
:1039C4003C20FCF721FC2D20FCF71EFC3DE7FEF714
:1039D400C9FC3BE70D4A80235B0011680B4313606D
:1039E400D4E62020FCF710FC43465F3B022B03D8AF
:1039F400684603F0A8F8C9E67B20FCF705FC202004
:103A0400FCF702FCC2E6C046446B00089814002090
:103A1400901400208C14002084140020FC01002049
:103A2400B414002064140020501400201008002056
:103A340010B5FFF79DFE074B1B68002B08D1064B02
:103A44001B681B789B00054A9B589847FEF706FEA7
:103A540010BDC046981400209014002000000020DF
:103A640010B51B4A1368013313601A4B1A68111DF1
:103A7400196019490B6853601A787F2313401B019E
:103A8400164AD3189B680B601B787E2B0BD8144AFC
:103A94001268032A04D09B00124A9B58984710BD11
:103AA400FFF7C6FFFBE70E4B1B68032B06D00E4B3C
:103AB4001B68002BF3D1FFF7D3FFF0E7FFF758FEA5
:103AC400094B1B68002BEAD1FEF7C8FDEFE7C0469F
:103AD400841400206C14002090140020100800208E
:0C3AE400FC0100200000002098140020CD
:103AF000F0B587B001AA3C4B13CB13C211001A6872
:103B00000A601B790B71394C394BE418394B1B682F
:103B1000A34263D2384D374E2F003BE0FDF720FF24
:103B20003FE0FFF79FFF28E0FEF70AFE00280CD1D8
:103B300033681B787E2B1BD82F4A1268032A14D0B7
:103B40009B002E4A9B58984717E0FEF701F9012881
:103B500008D00228ECD12A4A80235B0011680B436D
:103B600013603BE0FEF700FCE2E7FFF763FF04E0D1
:103B70003B68032B1FD0FFF775FF214B1B68002B01
:103B80002CD11C4B1B68002B1AD00133194A13602F
:103B9000A34223D22B68002BC6D11A4B1B68042BDF
:103BA000BCD0144B1B681B787E2BBAD89B00134AE1
:103BB0009B589847E1E7FFF7DDFDFEF751FDDAE797
:103BC0000D4B1B68032B0BD00B4B01221A600023FB
:103BD0000D4A13700D4A13600D4A136007B0F0BD13
:103BE00001A802F0B2FFEFE7046E00081002002007
:103BF000000E002090140020FC0100200000002096
:103C000098140020481400202B150020B014002028
:043C100084140020F8
:103C1400F8B5274B1C68002C2ED1264B1B681901C4
:103C2400254A5218D168C022120511420AD0234AEB
:103C34001168081D10601B011F4AD3189B684B6054
:103C44002000F8BD1B011C4AD3189A681C4B1A604B
:103C54001C4B01221A701C4D2F681C4C26685223E1
:103C64002B6023601A4B00221A60FFF73FFF2F607E
:103C74002660184B1C68E3E70E4B186802010E4BD4
:103C84009B18DA68C0231B0514001C401A4204D197
:103C940080231843FEF71AFBD2E76920FEF716FBD0
:103CA400044B1868FEF712FB0A4B1C68C8E7C046B1
:103CB4009C140020701400201008002064140020BC
:103CC400901400202B1500204414002040140020E0
:083CD400A01400209814002048
:103CDC0070B50023384A1370384A1360384A1360A1
:103CEC001500384E0EE0384B1B68FF2B24D868208B
:103CFC00FEF7E8FA344B1868FEF7E4FA304B1A6812
:103D0C002E4B1A60314C2B682268934230D2FEF74E
:103D1C0025F93378002BF6D0FEF7C0F900281FD018
:103D2C002B4B1B68002BDED12A4A1368191D11601E
:103D3C00254A12685A60E1E76720FEF7C3FA224C65
:103D4C0003202056FEF7BEFA0223E05EFEF7BAFA15
:103D5C0023681812FEF7B6FA2068FEF7B3FACDE71F
:103D6C00FEF746FA002809D0FFF74EFF002800D0D6
:103D7C0070BD134B1A68114B1A60C3E7FEF7FCF9C0
:103D8C0000280AD0FEF7B6FA134B1B68002BEFD1B4
:103D9C000B4B1A68094B1A60B4E70F4A01231168E0
:103DAC000B4313600D4B1A680D4B1A60044B1A68C9
:103DBC00024B1A60DCE7C0462B150020381400209B
:103DCC0040140020C01300203C1400204414002098
:103DDC009C1400206414002098140020A4140020CB
:043DEC00A8140020F7
:103DF000F0B5DE4657464E464546E0B591B00BA9B4
:103E0000B94B0A0013CB13C203CB03C206AAB74BAC
:103E100013CB13C211001A680A609A888A809B79B2
:103E20008B7102AAB24B13CB13C21B881380B14B08
:103E30001A68B14B1A60FEF797F8FEF7DFF9002811
:103E40000DD1FEF79FF9002805D1AC4A0123116876
:103E50000B43136018E10BA802F077FE14E1A54BA9
:103E60001A68A54B1A6006A802F06FFEA44D2B68D5
:103E70001801A44C001903F0F7F80D20FCF7C6F95F
:103E80002B681A01A418E168C0221205080010402E
:103E90000190114200D0FEE01B019A4AD3189C68A1
:103EA000994BE41A2405240D1B5D0125642B00D1D8
:103EB000D1E0954E24E00D20FCF7A8F9019D1FE00C
:103EC000914B1A195078000202341F5D07432820D5
:103ED000FCF79CF9781C03F091F82920FCF796F97F
:103EE00001352020FCF792F92020FCF78FF90134EE
:103EF000854B1B5D642B00D1ADE00135072DDAD871
:103F0000A0190004000C03F079F83A20FCF77EF9C0
:103F1000305DFFF7F7FB335D1A006B3A0A2ACFD901
:103F2000682B1AD0672B2ED0692B4CD06A2B57D018
:103F3000652BD6D12220FCF769F9734B1B195B78EE
:103F40009B46A31C98465B46002B7DD06E4B43449A
:103F500099465C460F239A466BE001342820FCF713
:103F600055F96A4B1B68102B08D0674B185DFCF79E
:103F70001DFD2920FCF74AF90135B2E7624B185DB7
:103F800003F072F8F5E76048021993781B04517842
:103F900009060B43D7783F020434025D13431F43E5
:103FA0002820FCF733F9594B1B68102B07D0380039
:103FB000FCF7FCFC2920FCF729F9013591E73800D2
:103FC00003F052F8F6E701342820FCF71FF94E4BB6
:103FD000185DFFF7BDFB2920FCF718F9013580E7D4
:103FE00001342820FCF712F9474B1F5D3800FFF71A
:103FF000AFFB3F01083743483F184020FCF706F964
:104000003804000C03F030F82920FCF7FFF80135E4
:1040100067E75C20FCF7FAF8380902F088FD5046A3
:10402000384002F084FD013C01239C46E144002C11
:1040300009D04B461F783B00203B5E2BE9D8380067
:10404000FCF7E4F8EFE7D8444446013C2220FCF7B3
:10405000DDF8033545E72C4820180004000C02F079
:10406000CDFF3A20FCF7D2F83B20FCF7CFF8244BE9
:104070001A681201234B9B18DA68C0231B051A42E9
:1040800009D10D20FCF7C2F811B0F0BCBB46B24616
:10409000A946A046F0BD02A802F057FD1B4B1B68C5
:1040A000102B18D0164B1A681201164B9B189868E3
:1040B00002F0F9FD2020FCF7A9F84020FCF7A6F853
:1040C0000F4B1868000108300E4BC0180004000C9C
:1040D00002F0CAFFD5E70A4B1A681201094B9B1878
:1040E000986802F0C1FFE5E7646B0008786B000890
:1040F0008C6B000840140020381400209814002015
:10410000701400201008002010020020501400201D
:10411000134B1B68134A1360134A126812011349A8
:104120005218BE20C000844661448A420AD2104917
:104130000139891A8908013189005118002001C20A
:104140008A42FCD10B4A934209D80B4A9B180B496F
:104150008C4662440021197001339342FBD17047B1
:10416000A8140020A41400208014002010080020AF
:10417000000E0020FE05000010020020FF050000D8
:1041800010B5164B1A68164B1A60FDF7EDFEFEF7D8
:1041900035F800280DD0114B1A68114B1A60114BDD
:1041A0001B68032B0BD8104A802311680B43136044
:1041B00004E00D4A212311680B43136010BD0B4A24
:1041C00013600B4A1B0100219954D318DB681B05AF
:1041D0001B0D084A1360FFF79BFFEFE74014002018
:1041E000381400207014002098140020801400203F
:0841F00010080020A8140020B3
:1041F80010B50023204A1360204A1360204A137028
:10420800204A1360204A1360204A01211160204A85
:104218001360204B1A68204B1A60204A002311783B
:10422800002903D0013310325F2BF8D11C4A1360E8
:104238001C4A1D4BD35C642B1CD01B4B1100013B4B
:10424800CA5C642A02D0002BF9D102E0002B00D00E
:104258000133164A1360FFF757FF154A154B1A60CA
:1042680000231360144A0F491160144A1360FDF7C4
:10427800CBF910BD0C4BEBE7A01400209C140020D8
:104288002B150020B014002084140020FC0100200D
:104298004C1400207C14002050140020100800202A
:1042A8008014002010020020FF050000A814002040
:1042B800F81200206C14002090140020981400209C
:1042C80030B5B9B036AAA04B196836919988918053
:1042D8009B79937134AA9D4B196834919988918080
:1042E8009B79937131AA9A4B03CB03C211001A88A8
:1042F8000A809B788B702EAA964B13CB13C22BAADD
:10430800954B03CB03C211001A880A809B788B70E7
:1043180027AA924B13CB13C21B88138022A9904B58
:104328000A0013CB13C203CB03C21CA98D4B0A008E
:1043380013CB13C203CB03C21B78137018AA8A4B82
:1043480013CB13C21B68136014AA884B13CB13C278
:104358001B8813800FAA864B13CB13C211001A684F
:104368000A609B888B8009A9824B0A0013CB13C271
:1043780003CB03C21B78137005AA7F4B13CB13C260
:104388001B78137001AA7D4B13CB13C21B881380B3
:104398007B4B1A687B4B54339A4200D280E07A49AF
:1043A8000423086803430B60764B0C339A4204D20B
:1043B800754A042311680B431360744B1B68002B68
:1043C8000FD0734B1968734B09010022CA545B184C
:1043D8005A709A70DA701A715A719A71DA719A6011
:1043E800DA606A4B00221A606B4B1B68002B0ED0F8
:1043F8000024694D2020FBF705FF01342B68A342F8
:10440800F8D85E20FBF7FEFE0D20FBF7FBFE36A872
:1044180002F097FB5C4C206802F0ECFD3D20FBF7B6
:10442800F1FE2368DB075ED4574B1B689B075ED4FD
:10443800554B1B685B075ED4534B1B681B075ED448
:10444800514B1B685B065ED44F4B1B689B065ED4C2
:104458004D4B1B681B065ED44B4B1B68DB055ED4BB
:10446800494B1B689B055ED4474B1B685B055ED4B4
:10447800454B1B681B055ED434A802F062FB464B13
:104488001868FCF78FFA2920FBF7BCFEFFF7B0FE8F
:104498000D20FBF7B7FE414B00221A6039B030BD42
:1044A800384B0C339A4200D282E7374B1B68002BFB
:1044B80000D082E7354B1B68002B40D1384B1B6876
:1044C800012BE5D02020FBF79DFE6F20FBF79AFE1D
:1044D8006B20FBF797FE334B1B68102BD8D1482075
:1044E800FBF790FED4E731A802F02BFB9CE72EA83F
:1044F80002F027FB9CE72BA802F023FB9CE727A8E8
:1045080002F01FFB9CE722A802F01BFB9CE71CA8FB
:1045180002F017FB9CE718A802F013FB9CE70FA812
:1045280002F00FFB9CE714A802F00BFB9CE709A81C
:1045380002F007FB9CE705A802F003FB9CE701A833
:1045480002F0FFFAA4E7C046CC6B0008D46B000861
:10455800DC6B0008E86B0008F46B0008006C0008CE
:10456800106C0008246C00083C6C00084C6C0008B7
:104578005C6C0008706C0008886C0008986C000877
:10458800641400205C130020981400209C14002060
:10459800801400201008002038140020B0140020D7
:0845A800A014002050140020B3
:1045B00010B500231B4A13600A221B490A601B49DD
:1045C0000A601B4A012111601A4A13601A4A1360DB
:1045D0001A4A073111601A4A2A311160194A1360C8
:1045E000013B194A1360194A1360194B31225624B2
:1045F0000021C02000051C705A709970D860996025
:1046000010330132D2B2352AF5D1124B313A1A6049
:1046100000230F493C328B540F4A1360FFF7ECFD27
:1046200010BDC046101500207C140020501400203E
:10463000FC010020B8140020581400206014002051
:104640005C140020941400207814002074140020BE
:0C4650001008002080140020A814002096
:10465C0070B5164C164D2B682360FDF77FFC2B684C
:10466C002360144B1D68013D28006B1C17D02D01D5
:10467C00114BED18114E10E08B420BD1002913D0C9
:10468C000132A95C935D1C00613C192CF4D8203BD1
:10469C00DBB2F1E7103D013804D30022F1E7012031
:1046AC00404201E00120404270BDC0463814002059
:1046BC00401400208014002010080020C01300209B
:1046CC0010B5FFF7C5FF0400431C0DD002011D4BB4
:1046DC009B18DA68C0231B051A420BD01A4A802398
:1046EC0011680B43136010BD174A212311680B434B
:1046FC001360F8E7FFF7ACFF431C11D00201114B1C
:10470C009B18DA68C0231B051A420FD1844213D9B7
:10471C000C4B24011C19A268000118188260E2E7F6
:10472C00094A212311680B431360DCE7064A8023F6
:10473C0011680B431360D6E7034A802311680B43BF
:0C474C001360D0E7100800209814002033
:1047580010B5FFF77FFF431C0FD003010D4AD21895
:10476800D3681B051B0D0C495B1892689A420AD343
:104778000001084A1018836010BD084A21231168F7
:104788000B431360F8E7054A802311680B43136055
:10479800F2E7C046100800201002002098140020FC
:1047A800F8B506000D490A68571C0F6054783F1980
:1047B800002C10D00D0005E05878FBF723FD013CD4
:1047C800002C08D02B685A1C2A60012EF4D0587887
:1047D800FBF70CFDF3E7014B1F60F8BD90140020B8
:1047E800074B1A68511C196051780902901C18600F
:1047F80092781143802292050A431A607047C04696
:0448080090140020E8
:10480C0010B5084B1B681B68002B08D0064A1368B0
:10481C0002331360034A1368043B136010BDFFF7A7
:0C482C00DDFFF7E764140020901400206A
:1048380010B5094B1B68191F1A680B689A4208D1F2
:10484800064A136802331360034A1368043B136073
:1048580010BDFFF7C5FFF7E764140020901400208F
:1048680010B5094B1B68191F1A680B689A4208DDB6
:10487800064A136802331360034A1368043B136043
:1048880010BDFFF7ADFFF7E7641400209014002077
:1048980010B5094B1B68191F1A680B689A4208DA89
:1048A800064A136802331360034A1368043B136013
:1048B80010BDFFF795FFF7E764140020901400205F
:1048C80010B584B001A8214B020012CB12C21B887C
:1048D800138002F036F91E4C2068FCF763F8236851
:1048E8001F2B15D00B2B1DD0194B1B68132B20D059
:1048F800174B1B68262B20D0154B1B68392B20D053
:104908003020FBF77FFC3020FBF77CFC04B010BDA7
:104918003220FBF777FC3520FBF774FC3020FBF7DF
:1049280071FCF3E73520FBF76DFC3220FBF76AFCDE
:10493800DAE73220FBF766FCDAE73420FBF762FCA3
:10494800DAE73620FBF75EFCDAE7C046B46C00080D
:044958002015002006
:10495C0070B5A6B0B54B1A6824929A886946942013
:10496C0009180A809B796A4696215218137022AD59
:10497C00AF4B2A0003CB03C2AE4B1A6820929A8825
:10498C006946842009180A809B796A468621521848
:10499C0013701CACA84B220043CB43C21B78137082
:1049AC00A64B1A681A929A881AAB9A80A44B1A686A
:1049BC0018929A8818AB9A8014AAA24B43CB43C284
:1049CC001B68136011AAA04B43CB43C20CAA9F4B8C
:1049DC0043CB43C211001A680A601B790B719C4BC4
:1049EC001A680A921A790AAB1A7106AA994B43CB28
:1049FC0043C21B88138003AA974B03CB03C21B78BB
:104A0C00137001AA954B19680191998891809B7933
:104A1C009371934B00934420FBF7F2FB6120FBF75F
:104A2C00EFFB7420FBF7ECFB6120FBF7E9FB24A800
:104A3C0002F085F88B480C3002F0DAFA280002F00C
:104A4C007EF824A802F07BF8874802F0D1FA200007
:104A5C0002F075F8854802F0CBFA20A802F06FF846
:104A6C00834802F0C5FA0D20FBF7CAFB814B1B688B
:104A7C00002B10D11AA802F062F814A802F05FF80B
:104A8C0011A802F05CF87C4B1B680024002B06D0AC
:104A9C00774E794D67E018A802F051F8EDE76E20DB
:104AAC00FBF7AEFB6F20FBF7ABFB6E20FBF7A8FB15
:104ABC006520FBF7A5FB0D20FBF7A2FBFFF7FEFE25
:104ACC006E4B1B6802229343012B02D00CA802F000
:104ADC0036F80D20FBF794FB0AA802F030F8684B6F
:104AEC001868FBF75DFF2C20FBF78AFB654B1B68F6
:104AFC00102B40D0644B1868FBF752FF2C20FBF7AF
:104B0C007FFB624B1868FBF74BFF06A802F017F807
:104B1C005F4B1E68002E3AD10020FBF741FF03A823
:104B2C0002F00DF85B4B1868002800DA70E0554B6A
:104B3C001B68102B00D16FE0FBF732FF01A801F0CE
:104B4C00FEFF554B1868002869DB4E4B1B68102B79
:104B5C0069D0FBF725FF0D20FBF752FB26B070BD8B
:104B6C00FBF74EFB01342B68013B1B01F318185D5E
:104B7C000028F5D19FE7444B186802F06FFA2C20FF
:104B8C00FBF73EFB414B186802F068FABDE7750174
:104B9C00AD1BAD00AD192D012900404802F088FA7B
:104BAC000400FBF7FDFE6643B404A41BA400A41B85
:104BBC00E400A4192401A41B6401394B9C466444F1
:104BCC002E20FBF71DFB2900200002F071FAFBF7E9
:104BDC00E7FE2900200002F0F6F98C00641864004E
:104BEC002900200002F064FA06002900200002F0DF
:104BFC00EAF9880040184000290002F059FA042311
:104C0C0083429B415B42F6183000FBF7C9FE86E7F6
:104C1C00684601F094FF91E702F020FA8EE76846AF
:104C2C0001F08DFF97E702F019FA94E7D86E0008AF
:104C3C00E06E0008E86E0008F06E0008006F0008D7
:104C4C00086F0008106F0008206F00082C6F000818
:104C5C00406F0008486F0008586F0008646F000828
:104C6C004F4646005C130020F81200201002002072
:104C7C001008002010150020B81400200815002082
:104C8C005814002050140020601400205C140020E4
:104C9C00941400207814002074140020006CDC02A2
:044CAC0000389C1C14
:104CB00030B58BB003A8124B020032CB32C232CBDC
:104CC00032C21B8813806A460E4B32CB32C201F0CF
:104CD0003CFFFCF77BF80028FBD0FF231840592845
:104CE00008D0684601F031FF0D20FBF78FFA002055
:104CF0000BB030BD0D20FBF789FA0120F8E7C04664
:084D00007C63000898630008C1
:104D0800F0B591B0040001A9334B0A0023CB23C2AC
:104D180023CB23C223CB23C203CB03C22F4D304E58
:104D280033682B60FDF71CF933682B60FDF7B8F981
:104D3800051E08D02B4A802311680B4313600025F9
:104D4800280011B0F0BDFDF719FA002804D10CA80D
:104D580001002A00244F0EE001A801F0F2FEFFF73F
:104D6800A3FF0028F3D10225EAE7002B12D0072A77
:104D78000AD001320131D35D0B701E00613E192E3D
:104D8800F3D8203B0B70F2E7164A022311680B4355
:104D98001360D5E70CAB1B78002B0CD0134A1268B4
:104DA800120113495218535501354378002B02D08C
:104DB8000130072DF7D10D4B1A6812010C4B9B18C7
:104DC8005D1900226A700B4A10680B4A82189A60B3
:104DD8002043D8600125B3E7A463000838140020F5
:104DE8004014002098140020C013002080140020D4
:0C4DF80010080020A81400201002002069
:104E040070B5C0200005FFF77DFF00280DD00A4CC7
:104E140022680A4803681D010949491915688D600B
:104E2400043A22600133036070BD064A012311680D
:104E34000B431360F8E7C04664140020801400207C
:084E4400100800209814002062
:104E4C0010B50020FFF75AFF002808D0022807D021
:104E5C00074B1A68074B1A60074B01221A6010BDEA
:104E6C00064B1B681B01064A00219954F7E7C04604
:104E7C00A8140020A41400209C14002080140020EE
:044E8C0010080020EA
:104E900010B588B06946214B0A0013CB13C213CB5F
:104EA00013C203CB03C21E4A13681C68043B136081
:104EB000962C1BD0112C26D0192C03D113240B2C8B
:104EC00018D002E0312C12D11F24132C12D01F2C29
:104ED00010D0262C0ED0392C0CD0602C0AD0114AC0
:104EE0008023DB0011680B4313600AE06024382C38
:104EF0000AD12624684601F028FEFFF7D9FE0028D3
:104F000006D108B010BD0B24572CD8D13924F1E7B5
:104F1000054B1C60FBF7ECF8F3E7C046D0630008D4
:0C4F2000641400209814002020150020CC
:104F2C0010B588B001A91B4B0A0013CB13C213CBCD
:104F3C0013C21B881380184A13681C68043B136047
:104F4C00164B1B68A34208D0154B1B68002B06D0D0
:104F5C00012C0DD813D0114B1C6008B010BD114A98
:104F6C00803311680B4313600C4B00221A60F4E77A
:104F7C000C4A8023DB0011680B431360EDE701A89A
:104F8C0001F0DDFD0D20FBF73BF9FFF78BFE002850
:104F9C00E1D1E2E7F46C000864140020081500204D
:084FAC002C14002098140020D1
:104FB40030B585B0174B1A6802929A8869468A817F
:104FC4009B798B73144B1A6800929A888A809B7918
:104FD4008B71FBF7C1FF114C23681D6802A801F017
:104FE400B2FDFCF729FD2020FBF70EF923681C68AD
:104FF400684601F0A8FDFCF71FFD2020FBF704F92B
:10500400FFF754FE002803D0054B1D60054B1C60C0
:1050140005B030BD6C6F0008746F00086414002084
:08502400BC140020141500204B
:10502C0030B589B001A80B4B020032CB32C232CB67
:10503C0032C21B68136001F082FDFFF733FE0028BB
:10504C0001D109B030BDFBF797FA034B01221A606E
:0C505C00F7E7C046F063000810150020C4
:1050680010B58CB006A91E4B0A0013CB13C203CB94
:1050780003C21B78137069461A4B0A0013CB13C27C
:1050880003CB03C21B781370174A13681968043BD3
:10509800136001290ED8002914D1684601F051FD8A
:1050A800FFF702FE00280BD0104B00221A60FFF712
:1050B8007BFA05E00E4A8023DB0011680B4313607E
:1050C8000CB010BD06A801F03CFDFFF7EDFD00286F
:1050D800F6D0064B01221A600120FBF7A9F8EFE78A
:1050E800246E00083C6E000864140020101500208F
:0450F80098140020E8
:1050FC00074B1B68002B09D0054B00221A60054A90
:10510C001368191D1160044A12685A607047C04632
:0C511C00B014002064140020AC1400202B
:1051280010B5214B1A68214B1A60FCF719FFFDF7DF
:1051380061F8002821D01C4B1A681C4B1A601C4BC4
:105148001A6812011B4B9B18DA68C0231B051A4208
:1051580019D0194B1B78002B1BD1184B1B68002B3F
:105168001AD117480368124A11680901114A5218DE
:1051780019689160043B036004E0124AA023116897
:105188000B43136010BD0F4A802311680B43136053
:10519800F8E7FFF7AFFFE0E76A20FDF795F8044B63
:1051A8001868FDF791F8EDE7401400203814002046
:1051B80070140020100800202B1500209C140020DB
:0851C80064140020981400207B
:1051D00010B50A4B1B78002B0DD1094A13680949F9
:1051E00018680860043B1360FDF75CFCFDF7E0FC09
:1051F000FDF738FD10BDFFF781FFEEE72B1500200E
:08520000641400209414002046
:1052080010B50D4B1B78002B0DD10C4A13680C49B7
:1052180018680860043B13600A4B1B88DB0705D538
:10522800FDF7C2FC10BDFFF765FFEEE7064B18223D
:105238001A60FDF733FCF3E72B15002064140020F7
:0C524800781400200004004094140020A2
:1052540010B50D4B1B78002B0DD10C4A13680C496B
:1052640018680860043B13600A4B1B88DB0705D5EC
:10527400FDF7F6FC10BDFFF73FFFEEE7064B1822E3
:105284001A60FDF70DFCF3E72B15002064140020D1
:0C5294007414002000040040941400205A
:1052A000F0B5C64600B588B069462B4B0A0013CB53
:1052B00013C213CB13C203CB03C2284B1B78002BA2
:1052C00014D1274A13688024A40519680C43043BB1
:1052D0001360244B9C420CD9234A8023DB001168C5
:1052E0000B43136008B080BCB846F0BDFFF706FF63
:1052F000E7E70D20FAF78AFF684601F026FC200058
:1053000001F07CFE270080370F25032398460FE02D
:105310000D20FAF77BFF200001F070FE3A20FAF72B
:1053200075FF300001F039FC00250134BC420ED07D
:1053300026780135102DEBD0300001F02EFC4346CD
:105340002B40032BF1D17C20FAF760FFEDE70D2015
:10535000FAF75CFFC6E7C0460C6400082B15002076
:0C53600064140020807F002098140020BE
:10536C0082B03A4B1A6801210A431A605A683848CD
:10537C0002405A601A68374802401A601A68364868
:10538C0002401A605A68354802405A60DA6A0F20A7
:10539C008243DA621A6B324802401A635A6B8A43B0
:1053AC005A6300229A60009201921968802252027C
:1053BC000A431A60190080229202A020C0010B68D7
:1053CC0013400193009B01330093019B002B02D1EE
:1053DC00009B8342F3D11D4B1B689B0306D5012315
:1053EC000193019B012B04D002B070470023019361
:1053FC00F7E71C4B11221A60144B5A685A605A6812
:10540C005A605A6818490A405A60596888225203EF
:10541C000A435A601968802252040A431A60190020
:10542C00802292040B681342FCD0084B5A6803216B
:10543C008A435A605A6801390A435A6019000C228F
:10544C004B681340082BFBD1CEE7C046001002403E
:10545C000CB8FFF8FFFFF6FEFFFFFBFFFFFFC0FFDE
:0C546C00ACFEFFFF00200240FF7FC0FFED
:105478004C4B80221A6000224B4B1A604B4908683B
:1054880080231B0203430B60494B1A601B68494A7F
:105498009A1849490A6049490A60494958184949C6
:1054A80008604949581849490860494958184949FC
:1054B80008604949581849490860494958184949EC
:1054C8000860494958184949086049498C46634465
:1054D80048490B60484B1B68002B06D11300183352
:1054E80046490B60464902330B6040231380354B15
:1054F8001B6800221A80354B1B6880211980354BA8
:105508001B6840491980354B1B6880204000188073
:10551800344B1B681A80284B1B689881DA8101304C
:10552800FF3018825A82314B1B681880314B1B6838
:105538001980314B1B68002B0BD1304B1B68C021E5
:10554800890019802E4B1B681A801B4B1B68998396
:10555800DA832D4B2D4A1A802D4B2E4A1A802E4B5A
:105568002E4A1A80244B1B68002B02D12C4B2D4A43
:105578001A802D4BBF2212021A6000232B4A136097
:105588002B4A13602B4A2C490A602C490A602C4A82
:105598002C490A602C490A602C4A13702C4A137053
:1055A8007047C0464C5C004034140020585C0040F2
:1055B800505C00400060004030140020F4140020CB
:1055C80002600040E014002004600040F81400204D
:1055D80006600040E414002008600040F014002039
:1055E8000A600040DC14002014600040EC14002025
:1055F80016600040D814002028140020E814002069
:10560800D41400200084FFFF005C0040203200001A
:10561800045C004031300000085C0040323000007B
:105628000C5C004033360000405C0040141400203D
:105638002C140020000E0020C8140020C4140020E0
:10564800CC110020D0140020CC140020011100201F
:04565800911200208B
:10565C0070B5204CE36980252D042B43E361FAF7E8
:10566C0035FD23691D432561FAF730FD236B80223C
:10567C00134323632369184A134023619022D205F4
:10568C00136816490B401360154B0021154A1980FD
:10569C0002339342FBD1144B0021144A198002337C
:1056AC009342FBD1124A116880231B020B431360F7
:1056BC00104C01232360C820FAF750FF002323600D
:1056CC00094A1360FFF7D2FE0B4B802212061A60B8
:1056DC0070BDC04600100240FFFF7FFFFFFF3FFC84
:1056EC00005C0040205C0040445C0040605C00407A
:0C56FC00585C0040405C004000E100E011
:1057080070B582B0284B1B68402B45D9274B1B68C6
:1057180040221A80244A1368403B1360234B1B68BD
:105728001B88002B16D0224C002122481F4D0368ED
:105738001E785A1C02605A780233036013023343FE
:1057480023800234013189B22B681B8801335B1036
:105758009942ECDB184B1B881B0604D5164A1388A4
:1057680016490B401380164B1B68164A1A80124BB9
:105778001B889BB26A46D380D3889B0602D40E4B03
:10578800114A1A806B4606331B88DB0602D40A4B83
:105798000E4A1A8002B070BD034B1968034A12689A
:1057A800118000221A60B9E714140020E0140020C8
:1057B8004060004020140020005C00400F8FFFFF75
:1057C800E41400200084FFFFA082FFFF9082FFFF07
:1057D80082B0174B1B6800221A80164B1B881B06C9
:1057E80004D5144A138814490B401380104B1B68C6
:1057F80000221A800F4B1B889BB26A46D380D3883D
:105808009B0602D40B4B0D4A1A806B4606331B8845
:10581800DB0602D4074B0A4A1A806B4606331B88FC
:105828005B0402D5034B074A1A8002B07047C04692
:10583800E0140020005C00400F8FFFFFA082FFFFF4
:085848009082FFFF80C2FFFF08
:1058500000B583B01C4A13881C490B4013801C4BB5
:105860001B68052B1DD01B4B1B68002B29D1164B29
:105870001B881BB2002B1EDB134B1B889BB26A4696
:10588000D380D3889B0402D40F4B134A1A806B46F3
:1058900006331B88DB0402D40B4B104A1A8003B07A
:1058A00000BD0F4B1B68802213430E4A1360084B48
:1058B00000221A60D7E7044A13880B490B40138073
:1058C000DAE7FFF721FFEAE7005C00400F8FFFFFF8
:1058D000181400201414002080A2FFFF8092FFFF04
:0C58E000341400204C5C00408F0F0000CE
:1058EC0082B0134B1A8813490A401A801B881B0676
:1058FC0004D50F4A138810490B4013800C4B1B889E
:10590C009BB26A46D380D388DB0602D4084B0B4A81
:10591C001A806B46DA8806331B889B0402D4044B2E
:10592C00074A1A806B4606331B8802B07047C04684
:10593C00005C00408F0F00000F8FFFFF9082FFFF75
:04594C0080A2FFFF37
:1059500030B587B0B74B1B881B0500D456E1B54A5C
:105960001388B5490B401380B44B1B78B4490B70B6
:10597000B44B1A78B44B1A70B44B1A88B44B1A80D3
:105980001A88120AB34802701B88DBB2B24A13703D
:10599000B24B1A88B24B1A80B24B1A88B24B1A809B
:1059A000B24B00221A60B24B1B68B24A1A800B78C5
:1059B000212B31D0A24B1B78DBB2A12B62D0A04BA4
:1059C0001A7861231A4206D09D4B1B78612213403E
:1059D000012B00D017E1974A138897490B40138099
:1059E000994B1A78D3B2062A00D17DE0062B66D8EF
:1059F000002B70D0052B00D0F6E09F4B00221A60E0
:105A0000FFF7EAFE924B1B887F2213409B4A1360EC
:105A1000964B05221A6005E18B4B1B78202B0BD08F
:105A2000894B1B78222B2AD1824A138882490B404A
:105A30001380FFF7D1FEF5E07E4B1B889BB2162248
:105A40006A44138013889B0402D47A4B8C4A1A80D0
:105A500016236B441B88DB0402D4764B894A1A80D8
:105A600016236B441B885B0403D5724BA022920063
:105A70001A80704A13881BB2002BFBDBD2E0FFF7C1
:105A800035FFCFE0704B1B78212B98D1694A1388E2
:105A900069490B401380784A07231360724B1B88B7
:105AA0009BB21268934204D26F4B1B889BB2724A1E
:105AB0001360754B754A1A60FFF726FEB2E0092B9A
:105AC00000D091E06C4B00221A60FFF785FE704B0E
:105AD000FF221A60A6E0684B02221A606A4B6D4AE8
:105AE0001A60FFF711FE9DE05A4B1B78012B1DD069
:105AF000584B1B78022B53D0564B1B78032B70D17D
:105B0000554B1B78012B69D15B4A17331360564BF9
:105B10001B889BB21268934204D2534B1B889BB2E2
:105B2000554A1360584B5C4A1A6028E0524B1222C7
:105B30001A605A4B1B68012B24D0594D524B1D60E3
:105B4000584B1C68584A012394421DD0681E6A466F
:105B5000D11CC25CCA540133132BFAD101AB1C72A5
:105B6000240A5C72514B9D4215D0514B1A7801ABFF
:105B70009A724F4A1268120ADA72434A1360FFF7A8
:105B8000C3FD4FE0494DD9E74A4B494A12689A4252
:105B9000F5D00123DAE7464B1A680332D2B2E6E7C2
:105BA0003E4B1B68012B12D0334B43221A60364BFD
:105BB000414A1A602C4B1B889BB22F4A12689342B1
:105BC000DDD2294B1B889BB22B4A1360D7E72A4BA7
:105BD00065221A602C4B394A1A60EBE7FFF786FE04
:105BE00020E0FFF783FE1DE0154B1B78002B02D051
:105BF000FFF77CFE16E00F4A13880F490B40138015
:105C0000FFF7EAFD0EE0FFF771FE0BE0094B1B8882
:105C10009BB216226A44138013881BB2002B03DB4D
:105C2000FFF7DAFD07B030BD1388034A1340014A7D
:105C30001380F5E7005C00408F0F0000806000409B
:105C4000261500208160004027150020826000405A
:105C50000211002028150020291500208460004032
:105C600024150020866000409212002018140020A5
:105C7000E41400200084FFFF1414002034140020DA
:105C800080A2FFFF8092FFFF20140020C06F000859
:105C90002C140020346D0008206A0008281400200D
:105CA000186D0008BC14002083040000446D000837
:105CB00014150020405700007C6F0008606E00083B
:105CC000F0B5DE4657464E464546E0B583B03C4B00
:105CD0001B881B0604D53A4A13883A490B401380A7
:105CE000394C0022394FB846394B9C46BA46B94622
:105CF00033E05346374E1E6044E001AB1B882B80D7
:105D00005A46354B1B681A802D4B1B889BB26A463E
:105D1000D380D3889B0602D4294B304A1A806B4625
:105D200006331B88DB0602D4254B2D4A1A8003B0AC
:105D3000F0BCBB46B246A946A046F0BD254B234960
:105D40000B600232D2B26B46598801AB1B88090244
:105D50000B432B80402AD4D00234A51E3B68214936
:105D600008688342CDD0694600264E8019788B465C
:105D700001A95E460E80013341460B606146096809
:105D80008B42B6D0531CDBB29B46402BB5D04B4662
:105D90001B6883420AD01878834668465E46468070
:105DA00001339942CAD009490B60CAE76B465A8849
:105DB00001AB1B88120213432B805A46CCE7C04626
:105DC000045C00400F8FFFFF02610040C4140020FC
:105DD00000020020000E0020DC140020A180FFFF44
:085DE0009180FFFFC8140020B0
:105DE80082B0114B1B881B0604D50F4A13880F4934
:105DF8000B4013800E4B1B6800221A800A4B1B882D
:105E08009BB26A46D380D3889B0602D4064B094AC4
:105E18001A806B4606331B88DB0602D4024B064AFF
:105E28001A8002B07047C0460C5C00400F8FFFFF1D
:0C5E3800D4140020A386FFFF9386FFFF18
:105E440010B5204B1B68002B34D01F4B186800285A
:105E54002FD01E4B1A681E4B1B689A4230D0511C1F
:105E64001A48016014781B4A1268914225D0174AD7
:105E74001268991A934201D2C433991A164B1B68BB
:105E8400002B11D07D290FD8134B00221A60134B1D
:105E94001B889AB29B0402D4104B11491980D30475
:105EA40002D40E4B0F4A1A80FAF708F98020000238
:105EB400204310BDFAF7F4FAC7E70B490160D6E7AF
:105EC4000020F6E70C1500202C140020CC14002030
:105ED400D0140020040200201C140020085C0040A0
:0C5EE40082A0FFFF8290FFFFCC11002085
:105EF00070B5634B19684A1C1A60012800D1B9E0DB
:105F00000A788B1C5E4C2360022800D1B4E04D78E7
:105F1000CB1C2360032800D1B0E08E780B1D2360DA
:105F20000438C0B2931E0D2B00D9A4E0052A32D04C
:105F30000F2A30D013000C3B012B3DD90423140051
:105F40009C43022C5AD0C978072A7AD84D4B00229C
:105F50001A704D4B1A68541C1C6015701A684B4B14
:105F60001B689A4269D0484B1A68541C1C60167012
:105F70001A68464B1B689A4278D0434B1A68541CE7
:105F80001C6011701A68414B1B689A4273D13E4BDA
:105F90003F4A1A606FE03B4B00221A703A4B1A6876
:105FA000511C196015701A68384B1B689A4262D1EF
:105FB000354B374A1A605EE0324B1B78AB420BD050
:105FC000314B1A68511C196015701A682F4B1B68E9
:105FD0009A420FD02B4B1D702B4B1A68511C196025
:105FE00016701A68294B1B689A4244D1264B284ADE
:105FF0001A6040E0244B264A1A60EBE7214B00224E
:106000001A70214B1A68511C196015701A681F4BC1
:106010001B689A420DD01C4B1A68511C19601670EF
:106020001A681A4B1B689A4225D1174B184A1A60F6
:1060300021E0154B164A1A60EDE7134B144A1A601B
:1060400091E7104B1B78AB428DD00F4B1A68541C54
:106050001C6015701A680D4B1B689A4202D0094BE0
:106060001D7080E7084B0A4A1A60F8E7064B084A99
:106070001A6082E7002070BD0020FCE70020FAE7EC
:106080002414002091120020D014002004020020CB
:04609000CC1100200F
:1060940070B582B0404B1B881BB2002B11DB3F4B09
:1060A4003F4A1A603F4B1B6818783F4B1B685A00E5
:1060B400D21890423FD940283DD83C4D374C260059
:1060C40025E0354A13883A490B401380E7E7FFF788
:1060D4000DFF14E0374B02221A600BE0364B1A68AE
:1060E400511C19603168097811701A68334B1B68A8
:1060F4009A421CD02368013323600138C0B22A4B72
:106104001B685A00D218904215D9402813D8012B85
:10611400DDD02B68022BE1D0204B1B681B78022BAF
:10612400D8D0042BDAD1234B04221A60E2E7224BA5
:10613400234A1A60DEE7234B1A681F4B1B689A42F6
:1061440020D99B1AC4339BB201AA13801E4B002290
:106154001A6001AB1B889BB27E2B18D80E4B1B8890
:106164009BB26A46D380D3889B0402D40A4B174A55
:106174001A806B4606331B88DB040BD4064B144A87
:106184001A8007E09B1A9BB201AA1380DEE70E4B2C
:10619400FF321A6002B070BD085C00402414002075
:1061A40000620040D81400202814002008150020A4
:1061B4008F0F000048140020D01400200402002097
:1061C400CC110020CC1400201C14002082A0FFFF5E
:0461D4008290FFFFB7
:1061D80000B585B0234B1A6801921B681B0429D5AA
:1061E800019A0F2313400393019A1023134002933B
:1061F800039B012B0BD0039B022B0BD0039B002B83
:106208000ED1029B002B08D1FFF71EFB1DE0FFF704
:1062180053FD1AE0FFF73AFF17E0FFF795FB14E08C
:10622800039B032B11D1104B1B68002B0DD1FFF7DB
:10623800D7FD0AE00B4B1B685B0508D4094B1B68AC
:106248001B050AD5074B094A1A6005B000BDFFF7C0
:106258000FF9044B064A1A60F7E7024B054A1A6021
:10626800F3E7C046445C004028140020FFF7FFFF16
:08627800FFFBFFFF7F80000027
:1062800070B5134B1B68002B21D0124B1A68511CA0
:10629000196010701A68104B1B689A4204D00F4E98
:1062A0000C4DAC24A4000AE00A4B0D4A1A60F6E734
:1062B000C02189008C466344991AA14207D9FAF794
:1062C000F1F832682B68991A9A42F6D9F0E770BD56
:1062D0002C140020C814002000020020C414002048
:0462E000000E00208C
:1062E400074B1B68002B00DBFEE7054A116880237F
:1062F4001B060B4313608369023383617047C046F6
:046304002CED00E09C
:10630800555342206173207669727475616C20431D
:046318004F4D3D00A8
:10631C0043466F72746820666F722053544D33324B
:10632C004630343220762E00202863293230323029
:10633C002D323420572E536368656D6D6572740071
:08634C00202D3E4442472000D1
:086354004B65726E656C3A00A6
:10635C00243100087A31000808320008083200089D
:10636C008C3100089E310008B0310008DC31000887
:10637C0020636F6E6669726D20772E757070657212
:10638C002063617365202759270000002063616E2C
:08639C0063656C6C6564200070
:1063A400205761726E3A2077696C6C206F76657243
:1063B40072696465204B65726E656C204F5020775E
:0C63C4002E73616D65206E616D65200018
:1063D000426175642052617465206368616E67650F
:1063E0007320696D6D6564696174656C7921200045
:1063F000536176652061637475616C20776F726B91
:0C64000020696E20466C617368203F002C
:10640C00313238205352414D2062797465732073B8
:10641C0074617274696E672066726F6D20307800DB
:10642C000000000000000000000000000000000060
:10643C000000000000000000000000000000000050
:10644C000000000000000000000000000000000040
:10645C000000000000000000000000000000000030
:10646C000000000000000000000000000000000020
:10647C000000000000000000000000000000000010
:10648C000000000000000000000000000000000000
:10649C0000000000000000000000000000000000F0
:1064AC0000000000000000000000000000000100DF
:1064BC0000000500000000000000000000000000CB
:1064CC0000000000000000000000000000000100BF
:1064DC0000000400000004000000000000000000A8
:1064EC00000000000000000000000100000000009F
:1064FC000000000000000000000000000000000090
:10650C000000040000000400000004000000000073
:10651C00000000000000000000000000000000006F
:10652C00000000000000000000000000000000005F
:10653C000000040000000000000005000000050041
:10654C00000005000000040000000400000004002E
:10655C000000040000000000000001000000010029
:10656C000000010000000100000003000000030017
:10657C000000030000000300000003000000030003
:10658C0000000300000003000000030000000300F3
:10659C0000000300000003000000020000000200E5
:1065AC0000000200000002000000020000000100D8
:1065BC0000000100000008000000080000000800B6
:1065CC00000008000000080000000800000008009F
:1065DC00000008000000080000000800000008008F
:1065EC00000008000000080000000800000008007F
:1065FC00000008000000080000000200000002007B
:10660C00000001000000010000000100000001007A
:0C661C000000050000000100000001006B
:106628004552524F5200000044524F5000000000A3
:10663800445550000000000053574150000000002E
:106648004F56455200000000524F54000000000011
:106658002D524F54000000005049434B00000000E9
:10666800524F4C4C00000000494E4A45435400002C
:106678002B00000000000000312B0000000000008B
:106688002D00000000000000312D00000000000077
:10669800414253000000000053484946540000009E
:1066A800414E4400000000004F520000000000006E
:1066B800584F5200000000004E4F540000000000E8
:1066C8002B2F2D00000000002A0000000000000011
:1066D8002F000000000000002A2F0000000000002A
:1066E8004D4F4400000000002F4D4F4400000000B3
:1066F80052414E444F4D00003D3D00000000000057
:10670800213D0000000000003E00000000000000E5
:106718003E3D0000000000003C00000000000000BA
:10672800553C0000000000003E3D00000000000055
:10673800303D000000000000564152434F4E00001B
:1067480052455600000000004B45593F000000002C
:106758004B45590000000000454D49540000000019
:106768002E000000000000002E480000000000007D
:106778002E440000000000002E220000000000004F
:10678800445A0000000000004858000000000000C3
:1067980052583F000000000052580000000000005E
:1067A80054580000000000004E545800000000003B
:1067B8005458220000000000584E4F5000000000BE
:1067C8004D5300000000000044530000000000008A
:1067D800544958000000000054494D45000000008D
:1067E800465245510000000050574D31000000004E
:1067F80050574D32000000004F48000000000000D4
:106808004F4C0000000000004950550000000000F7
:106818004950440000000000495A000000000000F0
:106828005244494E00000000524144430000000019
:10683800494E492D5350490053504900000000006B
:106848002E53000000000000465300000000000026
:106858004F505300000000005553455200000000FF
:1068680053454500000000004D454D000000000064
:10687800535400000000000052554E000000000074
:106888004E4F2D4442470000444542554700000002
:10689800464F52474554000041424F5254000000B1
:1068A8005245504C41434500524553544F524500C0
:1068B8004946000000000000434153450000000025
:1068C8003C434153450000003E434153450000000E
:1068D800454C5345000000005448454E0000000058
:1068E800444F000000000000554E54494C00000081
:1068F8005748494C45000000414741494E000000B7
:10690800464F5200000000004C4F4F50000000005E
:106918004900000000000000434F4E5449000000A9
:10692800425245414B0000005A425245414B00003B
:1069380052455455524E00003A0000000000000035
:106948003B00000000000000646F53545200000038
:10695800646F494F53545200646F4C49540000000F
:10696800646F4C4954384200646F56414C55450099
:10697800646F524556000000646F494600000000ED
:10698800646F434153450000646F3C4341534500E5
:10699800646F3E4341534500646F454C53450000C6
:1069A800646F444F00000000646F554E54494C001A
:1069B800646F5748494C4500646F414741494E0050
:1069C800646F464F520000004C4F4F5000000000CB
:1069D80052502D310000000052502D3400000000AC
:1069E8004155544F45584500424155440000000068
:1069F80053504C4954000000564944504944000043
:106A08003F00000000000000534156450000000010
:086A18004C4F41440000000056
:106A20001803430046006F007200740068002D00D8
:086A30004D004900440049003B
:106A3800FEE7FEE7FEE7FEE7FEE7FEE7FEE7FEE726
:106A4800FEE7FEE7FEE7FEE7FEE7FEE7FEE7FEE716
:106A5800FEE7FEE7FEE7FEE7FEE7FEE7FEE7FEE706
:106A6800FEE7FEE7FEE7FEE7FEE7FEE7FEE7FEE7F6
:106A7800FEE7FEE7FEE7FEE7FEE7FEE7FEE7FEE7E6
:106A8800FEE703488546FEF76DFC03E0704700000B
:046A980000180020C2
:106A9C0011488546114C20680434004201D08047CF
:106AAC00F9E70F480F49091A082903DB0022026095
:106ABC00043001600C480D49884205D0026804304E
:106ACC0003B4904703BCF7E700208646EC46002051
:106ADC000021074A9047FEE70018002024710008A7
:106AEC0030150020781600206D6D00086D6D0008C3
:046AFC00A10B0008E2
:106B000004207146084202D1EFF3088001E0EFF360
:0C6B10000980014908470000E562000808
:106B1C00756E646572666C6F77212000202D2D2DAB
:026B2C00200047
:106B2E0010B502003030C0B2392801D93732D0B298
:066B3E00F9F765FB10BD34
:066B44002849502D3E001F
:106B4A0010B5441C0078002806D0F9F75AFB013426
:0A6B5A00631E18780028F8D110BD62
:106B640063616E277420534545204B65726E656CD6
:106B74004F707300557365724865616465725F5345
:106B840074727563743D0000566172436F6E3A56B9
:066B9400616C75653D0017
:106B9A0010B5040003061B0F18003030392801D93C
:106BAA0037331800F9F72DFB0F200440200030304E
:106BBA00392800D90730F9F724FB2020F9F721FBFF
:026BCA0010BDFC
:106BCC004572726F722300002028636F6C200000E6
:106BDC00206E6F7420666F756E6400005F53796E63
:106BEC0074617820457272005F537461636B204549
:106BFC00727200005F436F6D70696C65206F6E6C14
:106C0C00790000005F4E6F20492F4F20436F6D6D50
:106C1C0020416363657373005F496E76616C6964D0
:106C2C0020436F646520616363657373000000002B
:106C3C005F6F7574206F6620436F6E746578740097
:106C4C005F52756E74696D65206F6E6C7900000013
:106C5C005F5468726561642063616E63656C6C651A
:106C6C00640000005F4E756D626572206F75742054
:106C7C006F662052616E6765000000005F446976A4
:106C8C002E6279205A65726F000000002020636F1D
:0A6C9C006D70696C696E672E2E00A2
:0E6CA60010B5F9F780FE2020F9F7ADFA10BD09
:0A6CB40042617564526174653D0091
:106CBE002F280FD90300303BDBB2092B08D90A2944
:106CCE000BD00300413B052B0AD83738C0B27047B2
:106CDE001800FCE701204042F9E701204042F6E7A8
:066CEE0001204042F3E723
:106CF4005553415254205465726D696E616C20671E
:0A6D0400657473206C6F7374210036
:0A6D0E0010B50120FBF7B7FD10BD22
:106D180012010002000000408304405724050000CF
:026D2800000168
:0A6D2A0010B50020FBF7A9FD10BD15
:026D340000005D
:0E6D360010B56B20FBF7C9FAFCF7A5FC10BDE9
:106D4400120100020000004083044357240500019F
:026D540000013C
:0E6D560010B56C20FBF7B9FAFCF795FC10BDE8
:096D640028566172436F6E3D0078
:0E6D6E0010B56D20FBF7ADFAFCF789FC10BDE7
:106D7C00203C2D6E6F742061204B65726E656C200B
:106D8C004F50206E6F722061206E756D62657200BF
:106D9C00203C2D696E76616C696420666F722042AE
:106DAC0061636B2D4374726C00000000203C2D520B
:0D6DBC00756E74696D65204572726F72000E
:0E6DCA0010B56E20FBF77FFAFCF75BFC10BDE6
:106DD80020202841444320696E697429200000005E
:0D6DE800202028414443206F6666292000CA
:0E6DF60010B57120FBF769FAFCF759FC10BDCF
:106E04002064656275672066696E697368656420CD
:016E1400007D
:0E6E160010B57220FBF759FAFCF749FC10BDCD
:106E24004C6F616420466C6173682050726F6A65B0
:106E34006374203F000000004C6F616420456D7056
:0D6E440074792050726F6A656374203F00FE
:0E6E520010B57320FBF73BFAFCF72BFC10BDCC
:106E600009026500020100803109040000000101EF
:106E700000000924010001090001010904010002C8
:106E80000103000007240100014100062402010162
:106E9000000624020202000924030103010201008A
:106EA00009240302040101010009058102400000D8
:106EB0000000052501010309050202400000000051
:056EC0000525010101A0
:0A6EC60010B50120FDF76DFC10BDB2
:076ED0006E6F2055534200D4
:106ED800537461636B3D00002052657475726E00D7
:106EE80020557365723D000020436F6465546872D5
:106EF8006561643D00000000456D70747900000014
:106F0800466C6173680000005F50726F6A65637455
:106F1800206C6F61646564002020204155544F4502
:106F280058453D002852533233323D5465726D69DD
:106F38006E616C29000000005350493D00000000BC
:106F4800202054696D65723A467265713D000000F3
:106F5800487A2050574D313D000000002C50574DC5
:036F6800323D00B7
:0F6F6C00564944203D200000504944203D20005C
:106F7C0009024300020100803109040000010202F1
:106F8C00000005240010010524010300042402075D
:106F9C0005240600010705830310004009040100C5
:106FAC00020A0000000705810240000007050202EA
:036FBC0040000092
:076FC00000C20100000008FF
:0A6FC80010B50020FDF7ECFB10BD32
:106FD2000A0010D00300400800E052008242FCD9AF
:106FE200002000E05208934200D39B1A40418A429B
:0A6FF200F8D1190070470020704725
:106FFC0010B50400000F16D12001000F17D120028C
:10700C00000F18D12003000F19D12004000F1AD142
:10701C002005000F1BD12006000F1CD10F20204093
:10702C00FFF77FFD10BDFFF77CFD2001000FFFF780
:10703C0078FD2002000FFFF774FD2003000FFFF70F
:10704C0070FD2004000FFFF76CFD2005000FFFF70B
:0C705C0068FD2006000FFFF764FDDFE771
:1070680010B504003020F9F7CDF87820F9F7CAF800
:087078002000FFF7BFFF10BD6F
:10708000CA1751408B1A17D0C1174A4004B4484060
:10709000411A48081A0000E052008242FCD9002040
:1070A00000E05208914200D3891A40419A42F8D137
:0C70B00004BC5040801A7047002070475C
:1070BC000A000FD00300400800E052008242FCD9C5
:1070CC00002000E05208934200D39B1A40418A42B0
:0870DC00F8D170470020704755
:1070E400CA1751408B1A19D0C11706B44840411A27
:1070F40048081A0000E052008242FCD9002000E057
:107104005208914200D3891A40419A42F8D10CBCEA
:1071140053405840C01A5140891A704700207047A4
:1071240055730008100200201C1300006B73000844
:10713400000000204471000810020000000000005C
:10714400F50E0008050F00082D0F00085D0F00085C
:10715400750F0008890F0008AD0F0008D10F000853
:107164001110000871100008D1100008ED1000087B
:10717400FD10000819110008291100084111000828
:1071840089110008A5110008C1110008DD110008CB
:10719400ED110008FD110008191200085112000831
:1071A40089120008C112000801130008191300080D
:1071B400391300086D13000891130008B513000873
:1071C400D9130008F913000859130008054E0008E4
:1071D400295100089D270008991900084919000839
:1071E400F51900083D1A0008251C00080F6D000859
:1071F4001D1400083D1400085D140008192A000835
:107204003D1C0008651C00082B6D0008B114000823
:107214005D2A00088D2A0008D9140008F514000816
:10722400D15100080952000855520008052E0008E3
:10723400752E0008E52E0008492F0008AD2F000820
:10724400652D0008A1300008CD320008093300087C
:107254005D1A000811160008B91C0008211B00085B
:10726400F13D0008A1520008311600083D1600083F
:10727400491600086119000881410008F941000815
:10728400CD46000859470008376D0008576D0008BF
:107294006F6D0008CB6D0008B524000815150008B3
:1072A400FD240008F76D0008176E0008536E0008EF
:1072B40029250008552500084915000891170008DC
:1072C4006515000879150008A11500084D4E000841
:1072D400AD250008C76E0008C96F000855160008E0
:1072E40095160008B5160008E11600080D480008B8
:1072F4003948000869480008994800080D17000833
:1073040031170008C1170008F917000861170008B1
:1073140031180008811800082919000839190008D3
:1073240079220008914E00082D4F0008B54F00083F
:107334005D4900082D500008695000080100000054
:107344000011002090120020C8110020006CDC0203
:10735400206861680834094204D0002202700130B8
:067364000139FBD1704766
:10736A0020686168A2680C34124205D00B78037059
:0A737A0001300131013AF9D17047EA
:0400000508006A8BFA
:00000001FF
